:020000040000FA
:2000000002013C8020FFFFFFFFFFFF8021FFFFFFFFFFFF8022FFFFFFFFFFFF8023FFFFFF30
:20002000FFFFFF8024301D03020EF402808D301D0302007A028519301D03020C4302800429
:20004000301D03C2AB3202CF79301D03C2AC3202CF7990BF32E04420F02290BF32E054DFC2
:20006000F022F4557E800C457E8008F4537EF85407457E90BF80F57EF022D5162E7516807D
:20008000C0D0C082C083D2D3FF90E002E06028FD758203E0C39D401474092007062004086C
:2000A0003007030245597449020A6F32200704E5617004E02405F0AE5D8E83758203E070B8
:2000C0001275825FE0602CD5E006F0200702D216F08020F583758202E030E517C2E5F07577
:2000E000820AE0600E758208D37D03E09400F00582DDF81EBEE0C2EFD083D082D0D032BD73
:200100001ABD1BB837B838B839B83AB83BB83CB83DB83EB83FB840B841B842B843B844E49C
:20012000F20890BF80E0F4540FF208E564F2089001377A0502E1BF440000060190BF32E0ED
:200140005406F090BFFE7430F090BF80E030E4030285B890BF32740630B5027402F0F075C2
:200160007E0090BF80E0F4540F23FE9000FF93CE049390BF36F00582EEF090BF34E4F0051D
:2001800082740930B502740BF090BF3374CFF0857D7C30B40A757C0090BF81E030E00343F2
:2001A0007E4090BF80E57EF090BF0474A7F0757D0075816612E6A6758164D21D7589017558
:2001C0008800759800D2B875A88290BF80E07B0020E70312E8E0E57E20E6030226051205A3
:2001E0001890BF35E020E73DBB00F30BB430EF1582E0B403E905827401F012051890BF35FD
:20020000E01582B44003022605B4420A7423F00582740202270CB44406E0F57B02E2DAB4CA
:2002200046BC023EE130E60A1582E0F00582E0F080F612E8E090BF35E0FF12050190E00A78
:20024000F0A3F0EF23C412050190E00CF0A3F090BF34E090E01AF0D20610E702C206700444
:20026000C206C21B90BF3AF0E57D60057D88020A7C90BF34EFF07D9005827410F030060765
:2002800090BF32E04440F012051890BF637403F012077775A0E090BF35E0F5147805F215CB
:2002A00082E030E004D21B54FEF51318F212331490E01AE090BF34F005827420F0300607F9
:2002C00090BF32E04440F01205187DA090BF34E0F51590E006F090E00AE024FF2323FB2547
:2002E0001354FEF510E5145303013BF511E5153BF512E5102404F54990E007F0E5113BF5DF
:200300004A0582F0E5123BF54B0582F090E00CE024FF23232549F546E54A3BF547E54B3BB4
:20032000F54890BF35E030E739E41582F00582F0793C90BF31E020E20AD8F7D9F5757D1525
:20034000020A7C90BF34E0FC0582E04C6003020A7990BF31E020E10AD8F7D9F5757D15020A
:200360000A7CF012338F7906D375A000E4F8FAF23308DAFB05A0D9F790BF20E4F005827441
:2003800000F090BF247401F0E513C37904301B02790899F533E5149400F534E5159400F595
:2003A00035793390E00CE0F5F090E00AE025F0500375370433500343370233500205375492
:2003C000FC301B0224042404F53675320BD2AA120B722000FD300806757D07020A7C75A0AB
:2003E0000012E1C9790412E1C7D9FB90BF20E4F005827400F090BF247403F07532097933D2
:20040000120B722000FD300806757D06020A7C75A000AA36AB3778000BBA00011B7480C38B
:2004200033FCE26C6006757D06020A7CEC0808D80205A0DAEBDBE990BF20E4F00582740413
:20044000F090BF247401F075320B7933120B722000FD300806757D07020A7C90BF32E04466
:2004600001F090BF34746630B50274D5F07DC005827440F030060790BF32E04440F090BF45
:2004800031E030E2F990BF32E054FEF090E01BE0F42401540790BF3BF090E01CE00314546D
:2004A0000FC4FB90BF34E0FF54FC60070324F1540F5002740F4B90BF33F4F090E01DF0EFE8
:2004C00030E121854DA090050B12E1E130B505782874D5F27820311F782AE57CF2784D7924
:2004E000561215AE90BF34E030E0FCD28C90E01AE06002D206855D62D2047539E1D2A880BD
:20050000205407FA74800A23DAFD221D011E0A28662904101812100090BF31E0F030E2FBA4
:2005200022300108C201D2027401116220004C10141BE55360057853020985E55560057827
:2005400055020985E5576005785702098520032BE559B55802802475A0E0A8591559B8104B
:2005600003755918E2F583F53975825F7403F0758203E0F5631219EF022D4EE551600312D9
:200580001634200015300212E54D700BE557600A7857794C1215AE0207F130070312463F11
:2005A0003017091207952007CF02064420030630180612073A0206442000FA3016F7E55950
:2005C000B5589474021162C210E562B55D0274E004F583F539758203E07045758231E0F5DA
:2005E000240582E0F5250582E0F5260582E0F527302112302904158380020583758203E015
:200600008539837031758201E0700F202B2875825FE0702285396202255A853962021ACABF
:20062000F563758212D210E030E00B8539621219EF1218D2A121E539B56290201006C216B1
:2006400074021167E54F60EC854F83C21075821CE030E705784F02097D758218E024E1F5BC
:20066000A07800790175821CE054F0700B7582027480F0E2F583807675821FE030E7327555
:2006800082027440F0E2F5836064758202E020E75D30E60AD210758201E0F58380EA1010FB
:2006A0004DE3B583F17903E3790170E8E54FF3803D758202E4F0758230E0FA0582E0FB0597
:2006C00082E0FC0582E0FDE2F5836022758202E054C0701A758230E0C39A0582E09B058218
:2006E000E09C0582E09D5006758201E080DAD216E27004E54FF2F3E58370097802E2FEE57B
:200700004FF28008758200E0FEE54FF0E583854F83758201F01582E0CEF06009F5830582D3
:20072000E54FF08003E54FF28E4FBE00048E4EA1218E83758201E4F0A12185603985605FAE
:20074000856083758203E0F5638560A0788690BF66E2F0080582E2F01219EFC2AF30400297
:20076000D200D20390BF637401F0752A02C218C2157412F0D2AF22D217C218C215C2039061
:20078000BF637402F0E4F078D579DC7A40D8FED9FCDAFAF022C2AF90E01EE090BF68F00585
:2007A000827405F090BF65749DF0E4300006C20090BF30F0D203F528F529C215C218C21AB1
:2007C000C213855D83758212E06006E4F0758203F0758286F075825F7402F00582F015839A
:2007E000E583B4E0E0200702D216C203D2AFC21722784D7949120AFD20E70AC202740112CF
:20080000006702052190BF207410F00582E54DF0F583120A4C3008057401020A6F854D835B
:20082000758213E06005740E020A6F758211E0700B1582E06006F5362414500C74ECF536E2
:20084000758210F00582E4F0120B992000FD3008057401020A6F7538027949120AD7ED30C5
:20086000E629E549B54607E54AB5470280177946753205120BBF3008057406020A6F90BFAD
:2008800039E030E7067538FC120AA3E549F5462404F549E54AF5473400F54AE54BF548346C
:2008A00000F54B90E00DE014F070161582E00582F090E007E0F5490582E0F54A0582E0F58C
:2008C0004B854D83758212E054F024D050057414020A6F30E4F830E503020521E561B40FAA
:2008E00005740A020A6F056190E003E4F0854D8375821CE0FB120C0BFD784D7A08604C549D
:20090000F00303FC758210E0C39C7A00403DED540F2323F0EB54F8700879501215AE0205CE
:20092000217904E475820BF0158274FFD9F9794E758219E0702F1582E0C395644027955C86
:200940005023255CF01215AE020521868375821C7480F0758210740CF075821E7401F005C0
:2009600082EAF08013868375821CE0D2E7F075821E7403F00582E4F075821DE4F079521247
:2009800015AE0205217913120AFD20E705D21402052190BF247401F090BF207410F005826B
:2009A000E6F08683B855028007B8531805171561C3E517940F4006F517740F8003E4C51793
:2009C000758212F0758210E02404F53675320B120A4C3008057402020A6F7538027913124F
:2009E0000AD7ED30E628E513B51007E514B5110280167910753205120BBF30080474068089
:200A00006E90BF39E030E7067538FE120AA3E513F5102404F513E514F5113400F514E51516
:200A2000F5123400F51590E00BE014F070161582E00582F090E004E0F5130582E0F51405CD
:200A400082E0F515794C1215AE02052175820FE0C2E0C39404F5331582E09400F534158292
:200A6000E0FC9400F5357933120B722000FD22F57D300701227D808003757D1375A89090D4
:200A8000BF34E57DF0FFA3EDF07407BF0901E412006B437E4090BF80E57EF090BF637403A1
:200AA000F080FE90E004E0F5330582E0F5340582E0F53590BF387401F00582E4F075320736
:200AC0007933120BBF300804740780A330060790BF32E04440F022301B0890E01DE090BF71
:200AE00033F090BF38ECF00582EDD2E6C2E7F0753207120BBF3008047407416F22C2433063
:200B0000190A90E01DE090BF33440FF090BF247403F090BF20740CF00582E6F07536047546
:200B2000370075320990BF3BE04418F0D20E75210090BF3CE72402F4F0058209E73400F487
:200B4000F009E73400120B812000FDC20E90BF3BE054E7F0200817868375820CE0FD20E732
:200B60000C301B0990E01DE090BF33F0ED227406416F75210090BF3CE7F0058209E7F00995
:200B8000E7543F20B50254035390C04290F57F30B50790BF32E054DFF090BF3EE536F42494
:200BA00001F00582E537F43400F090BF3BE054DF3043024420F090BF30E532D200F022E5C4
:200BC000385480600274FFFF30B50790BF32E054DFF090BF3CE72538F0058209E73FF00957
:200BE000E73F543F5390C04290F57F058274FEF0058274FFF075210090BF3BE054DFF090CD
:200C0000BF30E532D200F02000FD22B4580374BB2224D85002E42294D783220044453C77CD
:200C2000000000339B9B3300000000880088008300000000000000000000008888880000ED
:200C40000000008003020D6EC0D0C082C083C0E0D2D390BF31E030E108D2017402F0020D79
:200C6000BC1582E020E0FC0582E030E102D20154F3F030005EFA30E73712005AE57F300EDD
:200C80000C543F20B5025403601714800804543F20B50254035390C04290F57F7011200E17
:200CA0000EEA30E031E53D453E453F45407027EA20E42520E52090BF3BE030E506D20CD249
:200CC00008803DEA20E03930E70920080690BF30E532F0020DBCD209D208D390BF3EE0F4A4
:200CE0009400FA0582E0F49400FBEA253DF53DEB353EF53EE53F3400F53FE5403400F54053
:200D0000300303204005C200020DBC20084390BF23E004FAEC25434007F543B50A00400B13
:200D2000C39AF5431582E02543F543EC03C2AF304207C53CC3953C8002253CF53CD2AF30D4
:200D40004B03120E42E53D453E453F4540701FD20AC20D104B10104A0D304C55C24C43D037
:200D600018C2A8020EFC43D018C2A8020EF9201C21200FDB204B1B30180AE55FB56013C2DA
:200D80004C120764C2A8E53C204205B55E0A80027006D20DD2A880BBC20DD2A830450DC262
:200DA000457C0290BF21E02402F0A10B120DC57199304E0843D018C2A8020EF6D0E0D0834C
:200DC000D082D0D0323043047C028012AC3C20420AE55EC39C0CB50C004001EC23FC90BF0A
:200DE00020E0FA600DE4C39AFAE5435403FC74029CFCC3E53D9AF53DE53E9CF53EE53F946D
:200E000000F53FE54094004013F5408C378A36E5332536F533E5343537F53422E53D2AF52E
:200E20003DE53E3CF53E753F00853D36853E37E53624FFE5373401C2E0FC753D00753E00AB
:200E400080CD1215D8E4C39530FAE531547FFB74029B252EF52EE52F3400F52F12005A8518
:200E60005A83758224E02AF5330582E0352EF534FB0582E0352F543F5390C04290F57F43D0
:200E80000B1F44C05B2401500312005290BF3CE533F00582E534F0855A83758220E0C39A14
:200EA000F53D0582E0952EF53E0582E0952FF53F0582E09400F540500AE4F53DF53EF53F3D
:200EC000F5402290BF14E4F090BF24F0855F83758285E090BF21F0F54390BF24E55BF09093
:200EE000BF11F0F542EA90BF10F0F54190BF20F0753C0022800902149002103D020F5FC0AC
:200F0000D0C082C083C0E043D01890BF64E0FD0582E0FC30E7061207770215A330E60A3007
:200F20001505D21A0215A38000ED30E6028000EC30E202D21530E55B90BF637401F07444C6
:200F4000F0301507C215C2180215A3305004D248801920540A205207205310D249800C3062
:200F60004006E52154256026305416752A007583E0855882E55FF0E558B410037558191583
:200F800058C203304002C200121A840215A3D24C0215A330E310201518305010752A02908D
:200FA000E0217421F0EC02117302116AE544B407F4ED30E5067545090211645407B407E5A7
:200FC00030154B90BF67E0541FB402DD90E01FE0F890BF62E058F8E030E7305407F975832A
:200FE000E175826DE0B5181675828BE0B5190F758212E0B40408858360D2180215A3E5838D
:201000000583B55DDC75450602116402116190E022E0F814600515827421F0E87028752A91
:2010200010304019200816200A1330420DE53045316007053CD24A021592300DF890BF633E
:201040007412F002158FB4017E3028BF1582E0B426EB758223E0B403B20582E0B401AC05BE
:2010600082E07A057934B435004016F9A8F075F004A47A00942AC5F094000AC5F050F588F8
:20108000F00582E0B410004002740FF890BF67F0855F83758287F01582EAF090BF66F09057
:2010A000E0217421F0E545B4010302116A90E0277401F0A37403F0A37401F0A3E9F0A3E836
:2010C000F0754501021164B40214304FDD855F83758229782B7A0712E1AFC24F8053B403E0
:2010E0001A304F4D855F83758229792B7A0712E1B7C24F30403BD24B0215A3B4040E7404E3
:20110000F52A855F83758212F002116AB4072EE545B40102802F64066050E54554806014CE
:201120007583397582447402F0740690BF62F0F54502116A90BF637403F00215A3B4091E5D
:20114000E545B4011C90BF67E4F0855F83758287F074051582F0758237E0F545800C20E75A
:201160000975450790BF63741AF090BF637412F00215A320E4030215A3AF44ED30150A3073
:20118000E2295407F5440212DE305005752A02803730E511E54430E00B754506D24990BF4D
:2011A00063741AF0ED20540330521D20E11420E21120E00890BF67E060B0800690BF67E059
:2011C00060A875442002139420E40302128B5407C5445406700C30440302126C204D03BE80
:2011E00000030212DEE5445406602CBE021890BF63E4F000E0701E0582E0FA0582E06005F2
:20120000F8D25680121EEF20E00D90BF67E0541F60050212B6D25590BF13E004F9EB254212
:201220004007F542B51900400BC399F5421582E02542F542E52E2BF52EE52F3400F52F1E84
:20124000304012EF30E006EB03253C8006EB03C53C953CF53CE52B9BF52BE52C9400F52CB0
:20126000E52D9400F52D452C452B7007D24D532A1F806BBE016810550D305662C2568F443C
:20128000AD1AE8020F128F4402158F5407C54420E703B4021890BF60E0FA855F83758236AA
:2012A000E0C39AF0943850367438F08031204D2E20E12B20E228855F83758230EBF0780090
:2012C000EF20E00790BF67E0541FF890BF60E028F5300582E03400BE0202D2E7F531EF54BC
:2012E000066021E54454067027FE90BF14F090BF10E541F00582E542F090BF63E4F0E07013
:20130000FD0213E8E5445406602090BF10E0F541C24E90BF637401F0E0B401FCE4F0E0707F
:20132000FDE544FA232A90132A730213E80213E80213B70213A502139402139402136C901D
:20134000BF147403F090E021E0B42602742104F090BF10F0058274E0F090BF607401F0054A
:2013600082E4F090BF637490F002158FE545B4011690BF107427F0058274E0F090BF61E48D
:20138000F01582740580DB90BF62F090BF637410F002158F90BF60E4F00582F090BF637465
:2013A00098F002158F90BF147403F090BF107444F00582E55F80A1855F83758235E0F905D1
:2013C00082E0FA743829F090BF147401F090BF10EAF00582E55FF0743829C39A70010490F9
:2013E000BF60F00582E46162D24FE53045317003021490C24E300F030214BA204D9690BF77
:2014000014E4F090BF60E530F00582E531547FF0FA855F83758230E0FBFE3047167402B5B7
:201420002B11E4B52C0EB52D0B75826CE0FB1582E08001E4C3953090BF10F090BF13E00479
:20144000F9EB9A2542B51900400699FA1582E02A90BF11F0AB1EE531A2E7E4F530F531FE7A
:2014600090BF14E5447A0720E0027A05EAF090BF64E05406700B15827490F02044030E405C
:201480000302158FC390BF60E4F0EB0582F080DEC24E200F25204D20304047E54430E007B5
:2014A000E53CB55E408004E53C703A200808200A05D24E02158FD24D6194205318754506E5
:2014C00090BF63741AF0D24DD253855F83758244E4F0BE00DE90BF64E0540670D66194025C
:2014E00015693041D3BE00F790BF14E5447A0720E0027A05EAF030440C90BF617402F01562
:20150000827406616290BF60E4F07B06B52D09B52C06EBB52B005019E54430E00BEB0325AB
:201520003CB55E00402E8009EB03FAE53CC39A50237B0230471E7402B52B19E4B52C15B57C
:201540002D12855F8375826CE0FA1582E090BF60F0EA8001EB0582F090BF64E05406702F39
:2015600015827490F00EBE0126E4B52D0AB52C07EB2BB52B0050182041DEE54430E00AE570
:201580003C2BB55E0040D18006E53CC39B50C930511120440E30400B300D0853D0EFD2A852
:2015A000020C45D0E0D083D082D0D0D2A8328683758200E0F6F5A06007E4F07801F28003A3
:2015C00018F6F0758201E7F0F5A0A7836006E5837800F22209A78322301B58304055856380
:2015E000A07827E2604DFB90BF38E4F00582EBF090E0047A03793312E1B77538FA753207C9
:201600007933120BBF3008057407020A6F90BF317404F00582E04440F0757D0890BF31E0F2
:20162000757D1530E2F690BF34E070F00582E070EBF57D228551A0781CE2D077D077448044
:20164000F2901648C2E775F003A4730216600216D902173B0217CA79527851B1AE020521C7
:20166000E408F2B81FFA7904087A0412E1A17818E2C39564400A24E1F539C3E2955C4002A1
:2016800080D5853983758201E0C2106020F5A0F56379047814E267700F0908B908F775820C
:2016A00003E06563601080107800E280DE201027D210E54F80D5801F8563A0781CE2D2E7AF
:2016C000F2E408B824FA7818E22564F2781E7402F2201003121808C157E408F2B81FFA79C6
:2016E00004087A0412E1A17818E2C395644040955C503C255C24E1F583758202E0C2106098
:2017000025F5A0F56379047814E26770140908B908F778088551837582247A0412E18CC166
:20172000577800E280D9201006D210E54F80D08551A078247A0412E194C157781EE230E04C
:201740002A7818E2C395645001E4C3955C4004E4F28018255CFB24E1F583758288E0541FCB
:20176000B40304EB0480E3EB2564F27818E2C39564400C955C500824E1255CF53980057882
:20178000510209658551838539A075821D7A01123DD678887A1A12E18C78AA7A0C12E18CE3
:2017A000C1578539837822E25403FA75828CE054FC4AF008E2A2E4781EE282E20582E092D1
:2017C000E4F075827CE0C2E0F0227820E2600778517A0C02094B781D7A0312E1947822E293
:2017E00054F090E019F0F27825E26006E4F2F418800218E290E002F07478F278267A02128B
:20180000E19412011F02165778007901E3FBF5836005E2758200F0E2FA6007C583758201B9
:20182000F0E4F2E552F385635270058563538005F5A0E563F2853983758200E0B5630BEB54
:20184000F070070582F00582F022758202E0B56302EAF0758201E0B563EFEB6002F022EA1C
:201860007902FBF5A0E320E705AA03E270F4EAF02285398375827CE0D2E0F022E490BF24D0
:20188000F090BF20F0F53C782E7A04F608DAFC204002F521F529F54174FE8539A0204603CB
:2018A0007885E2F54290BF21F0F5437838E2C40354079019E793783520200104F2782B79A3
:2018C000297A0712E1A8121A3C752A0185395F121A847802E2D2E5F2301906C21975210029
:2018E0002285395FD20330401BD200204216200A13E53CB55E00500CC20DD2D3120DC512C8
:201900000B99C2D390BF637445F0101A06201703301506752A010219C3E0B445EA2050EAE3
:201920007401F0752A018539A0788AE20582F07837E2F54590BF147401F090BF11E539F0E8
:201940007437302001041582F07886E2703220280808F2187405F280277437F090BF61E4DB
:20196000F015827406F075A0E078279019E27A0512E1BF75450190BF637444F074C3802535
:2019800090BF66F0058208E2F090BF61E4F07835E21582F0243808F290BF637444F074C2C1
:2019A00030200274C17544FF304605201315D213F0101A0A2015072017042050F4223046A9
:2019C00002C213304005304205C200C20322D21CE521542560FAC21CC2003050EEC20302FF
:2019E0001A84010301340F060A0606060C060A85635A8539A0780FE2F521792808E2F70919
:201A0000B932F9793A08E2F709B943F97831E2F52408E2F52508E2F52608E2F527304033FA
:201A20007823E2F53208122AD090BF24E4F07827E290BF20F008E20582F0F543304014901A
:201A4000BF24E53220E107204304740780027405F0F55B7885E230400490BF22F090BF1252
:201A6000F030410720070424048004255E255E1430400490BF23F090BF13F074387836F299
:201A80008563A022855F8375820FE521F07828E60582F008B832F8783AE60582F008B84340
:201AA000F8304025758223E532F00582E533F00582E534F00582E57FF090BF20E0855F83C8
:201AC000758227F0E5430582F022853983758201E0758203F0F5A0F563F55A753A03781FAF
:201AE000E230E003753A01853A3B781CE2B458030222D1FA781DE4F2EA24E0403124104095
:201B000016901B0B540775F003A473021BB4021C6A021ED3021EEB901B1F75F003A473027D
:201B20001EF0021B22021F15021B28021FDE901B3675F003A4730220D802210602217C7844
:201B4000207A0412E1948039300F09781D7A0712E194802685398375826178207A0412E17A
:201B6000848017781FE4F2188006781E7401F208E9F2D0E0D0E080C77900E4781FF218E9D1
:201B8000F2781CE24480F27818E22564F2781DE285398330E70A75828178307A0412E1844C
:201BA000758203E4F07582067406F0C243C2051108020521853983758288E0B4030A781EEC
:201BC000F2058208E0F280B97404F0302E0C12293E122D3D1231D320E2F4781EE220E0042A
:201BE000E4F2809DE4F275828AE0FA0582E0FB7583E175828AE0B5020C0582E0B5030675C8
:201C00008288E0603CE5830583B55DE67583E175828AE0B5020D0582E0B5030775827CE0DF
:201C2000D2E0F0E5830583B55DE5117175828CE030E70C122934122D3D1231D320E2F461BB
:201C4000817960617A85398375828DE020E40420E5052274108002800DD000D000781FF2BA
:201C6000187406F2613F742080F3D205122938122D3D1231D320E2F420E411122959122D7F
:201C80003D122B9A600B20E2E330E0187903021EA7853983758288E0700A781EF208740156
:201CA000F2021EBB12367E6003021DE5753A03853983758285E0F5A012E1C91228BE122D53
:201CC0003D122B94600920E2E6D53AE3021D89302F03021DC2853983758285E0F5837582BC
:201CE00004E060E8C22DD22C753A03793F123DDD1228E2122D3D122B94601420E00E20E248
:201D0000EAD53AE7D22D102CDF021D89021C8C853983758285E0F5A07900E37009202D69BA
:201D2000C22CD22D80C2C210853983758285E0F5A07A08123DF6700B0808E230E00554FED5
:201D4000F2D2107A38123DF6700B0808E220E4054410F2D2103010317AFF123DF67800E291
:201D60000475825AF0F9E4F27802F2753A037B011228FE122D3D122B94600E85398375828A
:201D80005AE0F920E2E8D53AE5203036202F33853983853A3B8539A078767404F278A279A6
:201DA0006E7A0412E19A7428752B021229BB122D3D122B9A20E2EF607C30241E30E61B3083
:201DC000E5188539837582A9E4F01582F01582F01582E5395407F0021E4830E002818C209C
:201DE000E10330E314117175828CE030E706122934122D3D7943021EA754C06003D53BA63B
:201E0000853A3B853983758276E0D5E009781EE220E135021E92F07582B2E0F80582E0F94B
:201E200075826EE028F0A3E039F07902A3E03400F0D9F9A1A6853983758285E0F5A07800B4
:201E40007A047582A612E18C302E0C122942122D3D1231D320E2F48563A01217A23026458B
:201E6000742812238C701F853983758285E0F5A078007A0575827712E18C758277E060258D
:201E80001223F0B4FF1F20271C8563A0781EE220E113117175828CE030E706122934122D24
:201EA0003D79E5800279008563A0853983758289781FE4F0F2E9158218F2F075828A782053
:201EC0007A1412E1847582A2E82404F87A0812E1846181853983758288E070031217A2752E
:201EE0008288781E7A2212E1846181122CFA6178122CFA7528021230E37428122A90117C4B
:201F0000122D3D122E0E600B20E0E820E3F020E1E261486178122CFA7528021230E391457A
:201F20007B04758285E014F5A012E1C7DBFB8563A0122D3120441C742A122A90117C122DDF
:201F40003D122EBE600B20E0CF20E3F020E1C961486178853983782B7582727A0312E1AF61
:201F6000752800758285F0F58312307E7806E6F00582D8FAC210752B00752C02753A037438
:201F80003F30100274EA752802122A03122D3D122B94601820E0E820E1E5D53A03021FAA14
:201FA000122A4060DAC21020E2DA6148C2108539837582727A03C37802E0982010046002D0
:201FC000D210F078000582DAF030108575826E7A04D3E03400F00582DAF8C2108096122C68
:201FE000FA914520250B781E7401F208740CF261812024F28539837582A279307B04C3E08D
:20200000FAE39A058209DBF74005791C121B6A123DC87582387407F075825B79037A041267
:20202000E1B7758285E0F5837582007A03123DD67404F0758207C378307A047903E237F0C7
:2020400008091582DAF7753A02E4752802F52DF52C752B0212187C122D3D122B9420E2E910
:2020600030070122600F122D1330E503021C66D53AD7021FE685398375826E78307A0412DE
:20208000E18C853983758285E0F58312307E7806E6F00582D8FAC210752B00752C02753A8D
:2020A00003743F30100274EA752812122A03122D3D122B94601F20E2E830E503021C66D5B5
:2020C0003A030220CF122A40C21060D520E2D7122D13021FE6021B78122CFA75280D123064
:2020E000C97428122A9075320975212012187C122D3D122E0E600C20E0E120E3E920E1DBC4
:20210000021B48021B78853983758288E06003122D047528051230C97428122A9075320BB8
:2021200075212012187C122D3D122E0E601120E0E120E30620E1DB021B481218D280E77802
:202140001FE220E60D85398375828CE020E003021B781215D875280D1230C97428122A9013
:2021600075320975212012187C122D3D122E0E60DE20E00620E3E930E1BD809685398375BF
:202180008288E06003122D047528811230C9121C45122D313044030221FE742A122A90752C
:2021A000212075320912187C122D3D122EBE601120E0D520E30620E1CF021B481218D2800E
:2021C000E7781FE220E60D85398375828CE020E003021B781215D875280D1230C9742812EE
:2021E0002A9075320975212012187C122D3D122E0E60DE20E00620E3E930E1BD808A853989
:2022000083782B7582727A0312E1AF783075826E7A0412E18C122ACED219D24012187CD287
:20222000D3120DC5120B99C2D32000FD200850853983758285E0F583E5376402601BAB83C7
:202240007A02853682E53760011A2583F583E4F0A3B582FBDAF985038312307E7806E6F073
:202260000582D8FAC210752B00752C02753A03743F30100274EA752812122A03122D3D126F
:202280002B94601B20E00330E1022188D53A0302229C122A40C21020E2DA60D3021B48C2EF
:2022A000108539837582727A03C37802E0982010046002D210F078000582DAF020100221AE
:2022C000C175826E7A04D3E03400F00582DAF88093853983781DE2B44505752800802DB463
:2022E00046117528051230E3122ACE75212075320B8019B447117528811230E3122ACE75E7
:2023000021207532098005790C121B6A853983758239E054E0F978347582387A0C12E18CCD
:20232000758239E0541F49F012187C122D3D75825F7403F030210D302904158380020583A5
:20234000F08539833048057903121B6375824478307A0212E184304028300825122F5E75E4
:202360008261782479207A04C3E0FBE23BF308090582DAF53009057969021B7A7989021BDC
:202380007A304905790B121B63021B787B0080027B04F535122D5D75827D79047A0412E1F8
:2023A000B7123E44780475826E7A0412E1AFD212753304753403E535752B021229BB122DA4
:2023C0003D122B9A8539A0600820E2EAD534E78007C212E535B42A0F786E7A04D3E2340098
:2023E000F208DAF9D533CC122D7EE43012011422E420276B302668853983122D5D75827783
:20240000E0B40500505490240E75F003A47302241D0224300224700224DE02250F8539A077
:20242000786579787A0412E19A740112254170227533037878796E7A0412E19A7428752B7B
:20244000021229BB122D3D122B9A601720E2EDD533EA853983758277E4F0122D7E7401859F
:2024600063A022742A719070E9740212254170E2123DC87582387407F075825B79037A0402
:2024800012E1B7758285E0F5837A03758200123DD67404F07582078539A0787879037A0477
:2024A000C3E237F015820908DAF7753302E4752802F52DF52C752B0212187C122D3D122B66
:2024C00094601420E2E7D533E474FF122541122D7E74FF8563A022740312254170EB742874
:2024E000719070E57878796E7A0412E19A753303742A752B021229BB122D3D122B9A600808
:2025000020E2EDD533EA8170740412254170BA7533037878796E7A0412E19A7428752B0204
:202520001229BB122D3D122B9A600820E2EDD533EA8170E41225417090122D7EE48563A093
:20254000228539A07877F27885E2F58375820078777A0512E18C742A618C753A0275828527
:20256000E0700104758203F0F563F5A0122926122D3D1231D375828820E022602530E20DF7
:202580007401B53A0875825F7404F0806DD53ACDE0541FB4030280627423F0805D7403F08F
:2025A0008058E0541FB403527404F075827CE0C2E0F012367E90E019E030E73EE54D700B69
:2025C000E55760367857794C1215AE854DA07A40781012E19478107420F27818E539C39472
:2025E000E12564F2781C7440F2782075828A7A2812E184784D79541215AE85398375820371
:20260000E4F0020521E0F57C12E8E0E57D6003020A6F12331412338FD28CD2A890BF637428
:2026200003F090E00274FFF0E57E30E60EE57CC395644004955C400E02343A90E020E0F5D6
:202640007CC3955C50F2255C24E1F539854D6385635A854DA078217402F2D2AAE57E30E675
:20266000140226D77933120B722000FD20080122740B020A6F75A0E0782C9027137A221299
:20268000E1BF7842E57CF28563A090BF20742CF0058274E0F090BF247401F0E4F535F5342C
:2026A000F53790BF3374E0F075331475360875320BD164E57E444012007375330075340213
:2026C000753618D16475331A753400753602D16490BF31E030E3F912079585398375820360
:2026E000E563F012367E8563A07528051230E37428122A9075320B75212012187C122D3D9B
:202700001231D370E12008DE90BF35E4F0C2AF3007FD221800E0005F001800DF25000B6A45
:20272000F4FC0301800000C0150000C11568F40500070A00023026158539A07885E2F583E6
:20274000758200123DD6742A718C600122E42030FB753A048539A078A2796E7A0412E19AF3
:2027600078727A0212E194853983758285E0FF14F5A0E55E25E0FB12E1C7DBFB8FA075822E
:20278000A679007A0212E18475825A7402F0742A752B041229BB122D3D122B9A600B20E278
:2027A000EDBC010280030228371228A278B2E2B4030302284078A279047A0412E1A178AAB2
:2027C000E2FB123E6578B4E26076FB123E157B02123E15780479727A0412E1A87885E2F5ED
:2027E000837582007A04123DD68539A0787379047A0312E1A17F007B20123E545007123E80
:20280000448C037C00780479737A0312E1A8EB785AF2602C23F52B742A1229BB122D3D1249
:202820002B9A600E30E2088539A0785AE280E5BC01051228A280B2EC600312540B740122AD
:202840007A02853983758285E0F5A0758272E0C333500305A0C3F8E0F40413FC70027C8083
:202860007B03E4F208DBFC7480F208B8000205A0DCEEDAEA74013022045002740275825A66
:20288000F0752B02742A1229BB122D3D122B9A600620E2EDBC01A01228A2D53A02E4220218
:2028A00027678539A0786E79047A0412E1A1785AE2FB123E447804796E7A0402E1A8123DB9
:2028C000C87A1275823C7424F08048123DC87A258041123DC87A0375823C7480F075284220
:2028E0008034123DC87A1A302C07758239E04410F075823AE9F075823C74FFF08015123D3E
:20290000C87A15758239E04B302C024410F075823CE9F0752802758238EAF0E4F52DF52C88
:20292000752B0202187C123DC8752800758238E4F002187C780280027801791B8008780009
:2029400080027801791E123DC8E9758238F0E875823CF075280002187C853983752802E4C4
:20296000F52DF52C752B02302203752B04123DC87582387408F075823C7401F002187C2079
:20298000440330230122758238E0541FF075823BE0541FF8758239E048F075823CE0758239
:2029A0003AF075823DE075823BF0758240E075823CF0758241E075823DF0227528028539C2
:2029C000838539A0758238F0123DC8E4F52CF52D204412E52B30220830E1042402F52B037B
:2029E00003758240F0787175823AC37904E230220113F0058218D9F5302903122B7B317FEA
:202A000002187C8539838539A0758238F0123DC8E4F52D787175823AC37904E230220113A3
:202A2000F0058218D9F575823FE52C30220123F00582E52BF0302905122B7BC21002187C87
:202A400090FE02E0540FB4054490FE0CE0FA6424600DEA64207036E4F52BF52CD2E222909E
:202A6000FE00E020E70F90FE02E020E508E4F52BF52CF52E2290FE06E06012F42401F52B5C
:202A8000752C02302203752C04E4022A8F740122853983758238F00582E054E0F0E4302341
:202AA0000775823EF00582F0758241F0793375823AC37A04E330220113F0190582DAF53055
:202AC0002903122B7B122B2B317F20400122782490BF32E054DFF090BF3CE2F533F005824B
:202AE00008E2F534F0F908E2543F20B50254035390C04290F57F30B50D43011F44C0592470
:202B000001500302005222853983122B2B7803758238E075823D54E0700475823B18E0248E
:202B2000FFF01582E03400F0D8F822758238E075824020E50375823CC3302215E52C54FC0D
:202B4000452D7019E52C13F8E52B13C813C813800AE52C13452D7005E52B13701CC3E52D6C
:202B6000540113600574FF022B79C3E52C1375823FF0E52B13D2230582F0228539A0783D9E
:202B800075825BC37A04E0F9E239F2058218DAF68563A022753000753100E4FAFBFC8539C5
:202BA00083758260E06004E4F0801DE52954037074853983758244E0540A7009E53045317F
:202BC0006064022C9830E304740480598539A0783879457A0C12E19AE521F30978287A0206
:202BE00012E1A8E53CF309782B7A0312E1A878417A0212E1A875A0FE12E1C98563A011D258
:202C0000122D5D122D3D122D7EC213E4FAFBE52954037011758244E030E305122CCF80A8E3
:202C200030E1047408FA22E530240340F690FE02E0540FFC758200E0FB853983758269F043
:202C40000582ECF0EBC2E7B47020ECB4090040028073902C5825E073806F806D802A803891
:202C6000806380BF800880298049F0B4300261C820E6B020E5AD20E413540FB40002800819
:202C8000B404028003B4099B74108099540FB4070474208090B4012330241C90FE09E0B4C9
:202CA0003415853983758245E0541FB40809FC75826AF07460812574408125B4080280D8FF
:202CC000B40B0280D374808125122CCFE481258539A0784579387A0C12E19A790F7A0312B9
:202CE000E19A791C7A0112E19A79137A0312E19A79217A0212E19A0219EF853983758288B9
:202D0000E0700122781EF20582E008F2D0E0D0E0021B3F790320E00E792320E40920E30164
:202D2000221218717943758289E4F01582E9F080D3781FE230E405302502D24422853983A1
:202D4000758204D0E0F00582D0E0F0020521853983758205E0C0E01582E0C0E022D005D0EE
:202D600006853983758206E004F582D0E0F00582D0E0F0E582758206F0C006C00522D00517
:202D8000D006853983758206E0F582E0C0E01582E0C0E0E58214758206F0C006C0052230EC
:202DA0002546EB30E7428539A07865796E7A0412E19A753A03752B00752C02C210743E308E
:202DC000100274E87528125103B15DB13DB17E7194601820E2E720E612D53A03022DE8515F
:202DE00040C21020E2DC60D5740122853983758285E0F58312307E7806E06670EB0582D8C4
:202E0000F879088563A0781DE2543FF2E422300F057902740422200820E5295403453045EF
:202E200031FA758260E04AFA758244E0540A4A7008204D047107740822B15D719A20E26DA2
:202E40007010ECB40104EB20E70A300856122F5E800AB1133008131230407011796920097D
:202E6000387907200C367989802F122F75EA79686460602BEA794820E71F85398375826A44
:202E8000E0B4010F7C0179E81232061223F0B4FF20B121B19F600879E8123204D53B167F96
:202EA000048017204D0B71077F08022EBA7F0180067F0080057F021215D8B17EEF22300F0D
:202EC000057902740422200820E529540345304531FA758260E04AFA758244E0540A4A7098
:202EE00008204D047107740822B15D719A20E26220E61830E503021C667010ECB40104EBFC
:202F000020E70A300843122F5E800AB11330080E123040700C796920092579898021122FE0
:202F200075EA79686460601D794885398375826AE0B4010B1232041223F0B4FF19B12112F0
:202F40003204D53B157F04C1BA204D0A71077F08C1BA7F01C1B77F00C1BA7F02C1B7C385F4
:202F600039837582617820793D7A04E297F008058209DAF7228A07853983EB20E70B7A082C
:202F8000758261123DD602303A8539A078687583FE2410400DE4F218758201E0541F7A03DD
:202FA00080067582037A04E0F2058218DAF9853983C3302912786575825B7904E0FAE29A5E
:202FC000F2058208D9F6C3786579617A04E230220233F2F30908DAF58563A07830758261F3
:202FE0007A04C3E2F9E099F0080582DAF68539A07A0440197961C3E333F309DAFA786379E1
:20300000647A03E2F31819DAFAE4F38006758261123DD63025247582B4E0601E8563A07899
:203020001DE230E705D2E6F28010D2E7F28539A078817582657A0412E1848563A08F0222AD
:20304000122F75853983758262E0FC0582E0FD0582E0FE122F5E853983758262C3E09C05FE
:2030600082E09D0582E09E5008781DE2543FF2E422EEF01582EDF01582ECF074FF2274FF25
:20308000F9FAFBFCFDFE758200D210E07808C3C933C9CA33CACB33CBCC33CCCD33CDCE3361
:2030A000CE30E701B3501263061063051863041463035063023063013123D8D205820582E6
:2030C000D582C805831010C3227824E230E0057929021B6330B50C7826E254C0600579101C
:2030E000021B6AC378007920E330E0057949021B63F53D24FF09E3F53E3401C2E0F52B09C7
:20310000E3F53F38F52C09E3F54038F52D85398330471875826BE53DF07001D30582E53E92
:203120005401F070045002C247E52D452C452B7007D0E0D0E0021B7830223779007830E290
:2031400030E004D2457902E52B20E104E92380027402252BF52BE52C3400F52CE52D340094
:20316000F52DE9600D781CE2B4120201ECB4220201EC7582A21231C47582A2401075827DEA
:203180001231C475827D4005791C021B6AC37D00E52D13FCE52C13FBE52B13FA7830E23AF2
:2031A000FA08E23BFB08E23CFC08E23400FDE0C39A0582E09B0582E09C0582E09D50137996
:2031C0000C021B6A79307B04C3E0FAE39A058209DBF722E4FA853983758260E06006E4F006
:2031E0007408800AE52954037013758244E0FAB41803741022540A0330E0022407227B011B
:203200007C0080047C007B0220050790E019E020E40122781DE24420F290E00EE0FD2401AC
:20322000F00582E0FE3400F0E54D60E6C001854DA07A40781012E1947810BB0104741C8049
:2032400002743CF278127410F2856383781488827A0612E184EDF208EEF208EBF208ED4EE3
:2032600070047A0180027A00E53B146003430240EAF2781EE9F208ECF20812011F746630D0
:20328000B50274D5F2087404F2853983BB012878187A0212E194782C7582617A0412E18421
:2032A000C37B04782C856383758224E2FAE03AF2058208DBF680507818E22564F2782A7586
:2032C000828A7A0212E184782C7582927A0812E184E53A2401953B7837F2087582A67A04F1
:2032E00012E184758269E020E70D8563837582307A0412E18480087582657A0412E1849013
:20330000FE007A1012E184784D79561215AE8563A0D001227558108558597562E1E4F58C9A
:20332000F58A90E0027442F075168075170E75A0E179007B08789212011F90336E12E1E11E
:203340007892E92564F2789EF205A009DBE7754DFD754CE9854CA015A078007901E4AC4C2A
:203360000C05A0F2ECF3140CB4FDF6E4F322060688048D805F0298059902950094019A51B8
:203380009B109C649D25AC01AE01B203B50400123CBB90E01EE0540704F8748023D8FDF448
:2033A0000582F0855C3A7539E18539A07831E2F52408E2F52508E2F52608E2F527788AE2F7
:2033C00004FA748023DAFD786DF2788BE2448020200244407837F2C42354E07839F2903498
:2033E00000C082C08378BFE27895F21475F003A49033F473023405023405023405023405FA
:20340000D53AA9800302343F74E0855CF084C2E0FB03F55E7583E1758285AA5C7400F02B76
:203420000583DAFA74E0255CF55D90BF80E0F4540F600690E020E0F564227414020A6F307F
:203440002F03023631E527789A90345175F003A47302348A02346302346902346F023475D7
:2034600002347B7452F202348A745AF202348A745BF202348A745CF202348A7436F2087488
:2034800040F2087464F2087425F2302418787D79047A0412E1A13022657B02123E1578AAEA
:2034A000E223F2805978BFE264046052302134202931785B79047A0412E1A178AAE2FB1297
:2034C0003E65123E1505A0795B78047A0412E1A815A0785B7A0412E194EE54E04F6039D26D
:2034E00023803578B779047A0212E1A17E007F0078ACE2FB123E1578AAE2FB123E15EE542F
:20350000E04F6002D22330290F785B79047A04C3E2C797F70908DAF830261378AAE2FB307A
:203520002A092030061B78B47401F2123E547804797D7A0412E1A8202520E420300378AA67
:20354000E278A27A04F2E408DAFB30300B740178B5F278B2F208E4F2806578B4E260DB789F
:203560008DE4F2787D79047A0412E1A178AAE2FBC0E0123E657B80123E6578B4E2FB123E07
:20358000157B03123E44780479B27A0212E1A87B04123E15780479A27A0412E1A8D003C01F
:2035A00003123E6578A279047A0412E1A1D0E0C395F0FB123E44780479A27A0412E1A82053
:2035C000305378ACE225E0F5F0302406202A0375F01478AAE2A4FA30242A202A27E5F06092
:2035E0000BC39402501EC3EA94F45018E4FFFE7D017CF478AAE2FB123E65E5F060010C8C0B
:20360000F0EBA4FA78A2E22AF27A0308E235F0F275F000DAF678A2797DC37A04E2FBE39BBA
:20362000F20809DAF730300678A2E29401F2023676789A7428F2087422F2087465F20874A0
:2036400025F2787D8539837582A27A0412E18C7582A2E09401F0788DE24420F278AA7406B0
:20366000F208087404F208087401F2E478B2F20808F208F208F2123DDD05A0053922202FF1
:20368000108539837582BFE064046005E48563A0220582F0758231E054E1F524F00582E0C4
:2036A00054F9F525F00582E0F5260582E0F527122D5D302805758286E4F0753A0385398371
:2036C000758285E0F5A012E1C91228BE122D3D122B94600F20E2E6D53AE3122D7E740185F8
:2036E00063A022F8853983758285E0F5A0E2B40505D22F0236FFB4040A300733300430D241
:2037000030802C70D5300707300404D230D2267810903B3D123B3160147810903B46123BB0
:2037200031600A7810903B4F123B317004D22AD224123DDD7801E2548085398375828CF059
:2037400005827480F030070A78087582C17A1C12E18C302415202F617582AA7420F075823B
:20376000AC7401F0202A03023A2930077020306D30056A853983758285E02402F0F5A078C3
:20378000007A1412E194753A031228CB122D3D122B94601520E2F2D53AEF8539A07885E26C
:2037A000F5A078007A1412E194853983758285E0C39402F0F5A0302F24753A038539837581
:2037C0008285E0F5A012E1C978037408F2780A7402F290E02C740CF07B0002391FC22DD23C
:2037E0002C7804E27002C22C753A037900202C03302D0D793F30070830050520300279BF40
:20380000123DDD758285E0F5A012E1C91228E2122D3D122B94601620E2D1D53ACE102C06FE
:20382000102DC50236DAD22D80BE023A29F8853983758285E0F5A0E27009202DE6C22CD25A
:203840002D80A5302A293007E12030DE12E1C978047420F208740AF2087402F2780B741E92
:20386000F2780D7401F290E02C7410F002391F202C59202D563007057582C1E4F07582C039
:2038800030E00674027B03800474017B02F0780CE27582B6F008E2F9C4540F7582ACF0E92F
:2038A0005406037582B4F0E954017582BEF008E27582AAF078107582B77A02C3E29BF018B8
:2038C00005827B00DAF67811023A247A03123DF67074300706203003200503023982080802
:2038E000F20804F208E4F20804F208E4F208F2E82403F8E4F208F2087402F208E4F27AFF86
:20390000123DF67800E20490E02CF0E4F27802F208E2600B7809E4F2087402F208E4F275C7
:203920003A0390E02CE0F97B001228FE122D3D122B94600620E2EBD53AE8302F03023A29C4
:20394000302A03023A29753A03793F1228E2122D3D122B94600C30E2030236BAD53AEA0264
:2039600036DA853983758285E0F5A07A03123DF66010D2107582B47401F07582AA7440F09C
:20398000803DC210A9000808E2701408E2B4010F08E2700B08E2FB08E2700408E26004D203
:2039A000107B013030027B00EB7582B4F0E92408F8E2FD08E2FC0808E2C39B7582AAF07AEB
:2039C00004123DF6601A7582AC7414F07582B67402303001E4F07582B77A08123DD6804993
:2039E000E82405F8E27582ACF02010E0FB7E007F00C000123E95D0007582B63030027C0041
:203A0000ECF02030032403FC187582B7C3E29CF0180582E29400F0E82404F87A027582B924
:203A200012E18C087A0412E18C753A031228CB122D3D122B94605A20E2F2D53AEF202F6B98
:203A4000300729203026300523853983758285E0F5A02402F583E4F8F5827A1412E1847898
:203A6000007A04E2702B08DAFA20243F8539A078B779047A0212E1A1EC4D602F7E007F000D
:203A800078ACE2FB123E1578AAE2FB123E15023B24853983758285E0F5A078037A04790453
:203AA000E2F71809DAFA4E4D4C70030236DA302F0A75827D78047A0412E1AF7B01123E4443
:203AC00020242D7582B7E0FB0582E04B70227582AAE0FB7582B4E02BFB123E657582ACE043
:203AE000FB123E6578047582B77A0212E1AF80A17804E2F908E2420108E260AFB404073041
:203B000024A9D2228003B402A208E249709D8539A0202F1030240D7B20123E65123E1512E4
:203B20003496800312343F1539122D7EE48563A022E4936007FAE2A3086A60F622534D4FE4
:203B40002D4335303100524F2D353033304500546168697469203100524F2D3530333145F4
:203B600000E493700610100122A393FAA3E493A32EF875A000E2B9FF057442020A6F30E00D
:203B800003CC4BCC03CB2330E008CC75A001F309E4CCCBDAE180CA7B7F78007C007A08E286
:203BA000C3CC33CC30E701B3500363049D23DAF008DBEAECF42275A00112E1C9C2107B0179
:203BC000E4FCF97EE775A000EE2419FEF8E26022B41F07903C81716180EB903C02D21054A5
:203BE0000770010423F893C804938883F582716180D3903C0C7161EC75A001F37197F202FA
:203C0000E24F00003C0F3C413C673C41050000050008010802080306040805040602070831
:203C2000080809080A080B080C080D040E080F04100811081201130314031500081608172D
:203C4000000500080108020803060408050406020708080809080A080B080C010D030E039B
:203C60000F000810081100050008010802080308040805080608070308030900080A080B6F
:203C8000000500040106020803040400E493700610100122A393FAA3E493A3F9E47D01CCBB
:203CA00013CC50014DCD23CDDB09CC75A001E2CC087B08DAEA8539A0F380D175A00112E15C
:203CC000C912E1F07197F9E26960057441020A6F7539E075A0017800E208FC7B0805399004
:203CE0003D50918C79BFE3B41F1085395F7539E0903DBF918C855F3980E530E402D21054FA
:203D000007603BF3903D4623F993C904938983F582918C79BFE3798CB4030474808002E318
:203D200003F37931E330E1B57900E305A0F315A0D9F805A07932E3D2E1F30539809FC3E5E2
:203D40003994E1F55C223D823D533D833DA73D8305BF000831083208AA06AC08B704B80277
:203D6000B408B6085B085C085D085E08BC04BB08BA04B908BE08BD018C038A038B000833CF
:203D80000834000831083208AA06AC08B704B802B408B6085B085C085D085E018C038A0372
:203DA0008B0008330834000831083208AA087D087E087F0880038A038B000833083400042C
:203DC0001B061C081E042000853983758239E054E0F07A0A0582E4F00582DAFB2285398349
:203DE000758231E524F00582E525F00582E526F00582E527F0227800E204FB7803E2042818
:203E0000F8E2543FF26A600C08E22804F8B5030040EF740122BB010122EB8CF0A4FCAAF061
:203E2000EB8DF0A42AFDE5F03400FAEB8EF0A42AFEE5F03400FAEB8FF0A42AFF4005E5F0C3
:203E40006001D322EC2BFCED3400FDEE3400FEEF3400FF22C3EC9BFCED9400FDEE9400FE33
:203E6000EF9400FF22BB010122BF0006123E957F0022C004AC05AD06AE07123E95D007C01B
:203E800006C005C0047E00ADF0AC07123E95D005D006D00722780075F00074FF8BF084C528
:203EA000F004FA6B700305F0FAAFF0EE8BF084F9AEF0D2118FF0EEA428F8EE8AF0A4AEF066
:203EC0002D50010E8BF08428F8ADF0EE70E6101107E9FEECFDE8FC22AEF0ECFDE4C8FC80A9
:203EE000D312E8E0E57D6003020A6F90BF357404F012051890BF35E030E2F6D20775A0E080
:203F0000903F4012431330B508903FA212431F8006903FA612431F903FAB12431F74521223
:203F200042B2903FD212431712E4747408784EF27E0012432AD2A890BF637403F0023FE031
:203F40000A4469736B204669726D776172652D5265736964656E7420446961676E6F7374AB
:203F600069630D0A436F7079726967687420286329203139383820456D756C657820436F75
:203F800072706F726174696F6E20616C6C207269676874732072657365727665640D0A554D
:203FA000430030372F0031372F31003820636F6E74726F6C6C65722C206669726D77617280
:203FC00065207265766973696F6E206C6576656C200049502061646472657373203D200079
:203FE00075816475A0E012E1C9F608B865FBD21D123314D207740712006775A0E0784E745C
:204000000AF2126C4E7C01740412455460027C0E7D0E7E001246CA90405E12431312448AAB
:20402000740612455460030245E3EC1490403475F003A473024DFF024F33024FAD025D76A6
:2040400002501A0250300249DA02619C02628F02642D02653A02666D026E40026E422020B0
:2040600020202020202020202020202020202020202020202020202020202020204F70746D
:20408000696F6E204D656E750D0A2D2D2D2D2D2D2D2D2D2D2D2D2D2D2D2D2D2D2D2D2D2D30
:2040A0002D2D2D2D2D2D2D2D2D2D2D2D2D2D2D2D2D2D2D2D2D2D2D2D2D2D2D2D2D2D2D2D60
:2040C0002D2D2D2D2D2D2D2D2D2D2D2D2D2D2D2D2D2D2D2D2D2D0D0A3120202D20466F7206
:2040E0006D61742020202020202020202020202020202020202020202020202020202020DE
:2041000020203220202D205665726966790D0A3320202D20466F726D617420262056657258
:20412000696679202020202020202020202020202020202020202020203420202D20446111
:2041400074612052656C696162696C6974790D0A3520202D20466F726D61742C2056657235
:204160006966792C202620446174612052656C696162696C6974792020203620202D2052DC
:20418000656164204F6E6C790D0A3720202D204C697374204B6E6F776E20556E697473203C
:2041A00020202020202020202020202020202020202020203820202D205265706C616365FE
:2041C00020426C6F636B0D0A3920202D2057726974652052435420202020202020202020A3
:2041E0002020202020202020202020202020202020203130202D204F70746963616C205273
:2042000065616420616C6C204469616720536563746F72730D0A3131202D204F707469639E
:20422000616C2057726974652061204469616720536563746F7220202020202020202020A0
:204240003132202D204973737565204D6F64652053656C6563740D0A3133202D2044697358
:20426000706C6179204E6F7672616D20202020202020202020202020202020202020202055
:2042800020203134202D2045646974202F204C6F6164204E6F7672616D0D0A0A456E746557
:2042A00072206F7074696F6E206E756D6265723A20001242B6E4C083C082F5F090BF34F005
:2042C000A37401F012051890BF35E020E02C30E1F390BF34E0547FB4030790E030E0440259
:2042E000F090BF357402F012051890BF35E020E1F690BF35E4F0E5F080C290BF35E4F0F59E
:20430000F012051890BF35E020E1C620E0F3D082D08322740A51B6740D51B6740A51B6E423
:2043200093600551B6A380F7808CE48007E47D007E007F00C001C0E075A0E078437A0B12E7
:20434000E194784EE2FB7843C000123E65E5F0D000F208EF70F2EE70EFED70ECEC70E9D07A
:20436000E02443FB944E4008742051B61BBB4DF8784D18E27010E86443600BC3E89B50F25A
:20438000742051B680ECB40A0040022407243051B618E2B842F0D001E441B612051890BF82
:2043A00035E030E1F690BF34E0547FF5F0A37402F012051890BF35E020E1F690BF35E4F0DB
:2043C000E5F02274081245497837E4F2719BFABA7F227837E260F574081245547004745C93
:2043E00051B67837E214F22438F8E251B2740812454380D8740812455460097408124549CC
:20440000745C51B6BA0D1D7837E2603BF5F07838E2B441004008B45B0050032420F208D58C
:20442000F0EE8023BA030B740112454390445C711F22EAC39420500280927837E2C3940A8B
:2044400050F612444780857837E204F2142438F8EAB40D01E4F27002740D41B25E4300C3B9
:204460008504F01244758505F01244758506F01244758507F0E2C5F095F00822C3E29C0862
:20448000E29D08E29E08E29F082271C312463FE4FCFDFEFF90E0387406124549740B124525
:2044A00049E07027740B12455470031244BD784F915F4004917C50127406124543AB0178EA
:2044C0005779047A0412E1A1A90322FA740B124543EAC3943040E1FA784EE2FBB41016EA22
:2044E000B40A00401EB4310040CEB4370050C9C39427FA800EB40805EA94088004EAC39497
:204500000A50B5A802123E15AB00123E44A3809171C312463F7838E26011F5F008E260028B
:20452000D322E5F0B4790122B46EF5C32275A0E075F008842430F8748005F023D5F0FCF571
:20454000F0E222B12D45F0F222B12DC5F0F4C5F055F0F222B12D55F02290E030E04404F0AE
:2045600020E30EC28CE58124FDF87445F6187479F6EFD083D082D0D032904581711302452C
:20458000DF54696D656F757420686173206F6363757272656420647572696E67206F706575
:2045A000726174696F6E00C28C75A0E0227402B14990E003E4F07582027442F0D28C2290A3
:2045C00045C67113619B48697420616E79206B657920746F20636F6E74696E75652000B101
:2045E000A7B1BFB1A7023FE09045F77113B11040F7B479012280EC44617461206F6E20642C
:20460000726976652873292077696C6C206265206C6F73740D0A446F20796F752077616ED2
:204620007420746F20636F6E74696E7565205B59206F72204E2C6465663D4E5D3F20009009
:20464000E030E020E05820E14390BF31E030E24E719BB403499046A47113780079007A1584
:20466000E52A602430180FC000C001C00212073AD002D001D000D8E8D9E6DAE490BF6374E4
:2046800003F03017FD1207957401B143740CB154600DA88190E036E0F6158218E0F622127C
:2046A00048E5A1E350726F63657373696E67205E4300784FC0017904E7F20809B908F9D0F2
:2046C00001227A04F2E408DAFB2275A0E0784FC002ECD1C2EDD1C2EED1C2D00222E539C391
:2046E00094E12564FC612D75A0E0786A746BF2F8E260040820E4F922D13F853983758231AC
:20470000E0F5240582E0F5250582E0F5260582E0F527D2A8B1AD122938122D3D1231D3201D
:20472000E2F27409B149753A0AB1AD122926122D3D1231D3601320E2F0D53AED7409B14352
:20474000740AB1547012024957122959122D3D1231D320E2F412367EA1A7853983758288C8
:20476000F01423F5F090477B93C5F0A393F58285F0837113904795711FC1DD47A047BF479C
:20478000E747FC4815482E484B485F4870488A489E48B548CF206F6E206472697665200007
:2047A0004472697665206E6F74207265616479206F72206472697665206572726F72004490
:2047C00072697665206572726F7220647572696E6720726561642F7772697465206F7065B6
:2047E000726174696F6E004F7074696F6E206E6F7420737570706F72746564005265706CA9
:20480000616365206F7065726174696F6E206661696C6564004572726F72207772697469A0
:204820006E6720524354206F722046435400536373692073656C656374696F6E2074696DBA
:20484000656F7574206572726F720053637369207472616E73666572206572726F720045AB
:2048600072726F72206F6E20636F6D6D616E64005370756E646F776E206572726F72206F40
:204880006E20636F6D6D616E640057726974652070726F74656374206572726F7200496E7E
:2048A000717569727920636F6D6D616E64206661696C6564004D6F64652073656E73652057
:2048C000636F6D6D616E64206661696C656400466F726D617420636F6D6D616E6420666125
:2048E000696C656400796B75A0E0E37001220954EF202FF3F539F583758288E06006124779
:204900006185398375829CE0FCA3E0FD450460D7C004C00590492E1243131246DD9049532D
:2049200012431FD005D0047E0012432A80B94E756D626572206F662062616420626C6F63BF
:204940006B7320666F756E64206F6E2064726976652000203D20007401802E7402802A74B2
:20496000038026740480227405801E7406801A74078016740880127409800E740A800A74A3
:204980000B8006740C8002740D12475A90E06AE014F582E04410F09049AC1243131246DDC5
:2049A0009049B312431F7405124543224472697665200020686173206265656E2072656D2E
:2049C0006F7665642066726F6D20667572746865722074657374696E6700D2057A0875A0A9
:2049E000E012E1C7DAFB12331412338F120795755E5FE54DF563F55AF5A012E1C9740A1281
:204A000045431246E7904B031243137539E00539853983758203E563F0758288E4F0758200
:204A20009C7A02123DD67582857400F01246F874091245546003024A64E539C394E12564EF
:204A4000FC905193124317740312432E904B4412431F8539837582A27A03790412E1B774FB
:204A60000E124334E539655D600280A23005030245DF904BA51243131246E76013124BD610
:204A80001246DD124BD66008904BB912431F80F0E564FC255D14FD1246CA904B531243133E
:204AA00012448A740B124554700B1246E76013740A1245492274061245546008904BBC1249
:204AC00043134105ECC3956424E1F5391246F874091245546008904B8812431380E4796B6C
:204AE000786AE2F8696009E3653960D6E80980F4E539F208E4F2E8786AF2741112455470C2
:204B0000AE80BF44726976652020205374617475732020202020202020556E69742053694E
:204B20007A650D0A2D2D2D2D2D2D2D2D2D2D2D2D2D2D2D2D2D2D2D2D2D2D2D2D2D2D2D2D93
:204B40002D2D2D002020202020417661696C61626C6500456E7465722061206472697665F4
:204B6000206E756D62657220746F20746573742028656E6420776974682052455455524E4E
:204B8000206B6579293A200044726976652073656C6563746564206973206E6F7420757351
:204BA00061626C650053656C65637465642064726976652873293A20002C20004E756D6202
:204BC000657220656E746572656420697320696E76616C6964007405124549786AE2F8E23D
:204BE0006026F539E804786AF2E53920E4EF853983758231E0F5240582E0F5250582E0F5F1
:204C0000260582E0F5277401227C017DFF7E011246CA785474FFF2904C3C1243131246DDD4
:204C2000904C6212431F12448A740612455470D98539837582A6ECF0EDA3F022456E74658C
:204C40007220766F6C756D652073657269616C206E756D62657220666F7220647269766540
:204C60002000205B312D36353533352C6465663D315D3A20001245E831DC1246E771D67071
:204C8000012220300291097C0020244D853983758232E020E1E7E583655D601B0583E03089
:204CA000E115AC8390E06BE07009904D621243130245DFA36C70F07C007D1F7E011246CAA6
:204CC000904D941243131246DD904DEF12431F12448A740612455470B3853983758277ECC3
:204CE000F02024992030967582BFE0B4048F907CCE124313907CC812431F7C007D038539E0
:204D0000837582B4E0FE1246CAAC0612432D907CC412431F12448A740612455470D08539EA
:204D200083758278ECF06033907D5A124313907CC812431F7C027DFA8539837582B6E0FE3A
:204D40001246CAAC0612432D907CC412431F12448A740612455470D0853983758279ECF0E7
:204D6000817D4D75737420616C736F20666F726D617420326E64206C6F676963616C206471
:204D800072697665206F662073706C69742064726976650030203D20646576696365206441
:204DA000656661756C7420696E7465726C656176650D0A31203D206E6F20696E7465726CD3
:204DC000656176650D0A456E74657220736563746F7220696E7465726C6561766520766127
:204DE0006C756520666F722064726976652000205B302D33312C6465663D315D3A2000915F
:204E0000751246E7757C0071D6700F740F124554700511E50245DF024F3A904E381243135F
:204E20001246DD125467740512455470D7904E521243171246DD80CC5374617274696E679C
:204E400020666F726D6174206F6E2064726976652000436F6D706C6574696F6E206F662023
:204E6000666F726D6174206F6E20647269766520002026098539837582B4E0601874071232
:204E80004543904E9612431312451040F5B46E05740712454922446F20796F752077616E18
:204EA0007420746F207265706C6163652062616420626C6F636B73206F6E20647269766563
:204EC000287329205B59206F72204E2C6465663D595D3F20007C017DFF7E011246CA904EA6
:204EE000F412431312448A740612455470E77868ECF2C171456E746572206E756D62657263
:204F0000206F66207665726966792070617373657320666F7220746865206472697665280E
:204F20007329205B312D3235352C6465663D315D3A20001245E831DCD1D51246E7757C01BD
:204F400071D6700F7412124554700511E50245DF025DA9904F741243131246DD12546712F2
:204F6000463F740512455470D4904F8E1243171246DD80C95374617274696E672076657234
:204F8000696679206F6E2064726976652000436F6D706C6574696F6E206F6620766572698D
:204FA0006679206F6E20647269766520009175D1D5740F124543C1017C007DFF7E01124661
:204FC000CA904FD612431312448A740612455470E7EC7869F222456E746572206E756D62DD
:204FE0006572206F662072656C696162696C6974792070617373657320666F7220746865B4
:20500000206472697665287329205B302D3235352C6465663D315D3A2000124C75124ED596
:20502000124FB8740F1245437412124543024E011249DC124E711246E774131245437407E6
:2050400012455460081245E87413124549757C02124BD670061248E50245DF90507C124325
:20506000131246DD12546712463F740512455470DC9050991243131246DD80D15374617213
:2050800074696E672072656164206F6E6C79206F6E2064726976652000436F6D706C657495
:2050A000696F6E206F662072656164206F6E6C79206F6E2064726976652000853983758288
:2050C0006E79047A0412E1B7740E124554700A90E9007404F0A374E9F07A007BE990E900EE
:2050E000E0F8A3E0B4FE06740112454322F9EA2404FAEB3400FBB50123EAB5001F8A828B1F
:205100008378047A04E6F008A3DAFAA883E58290E900F0A3E8F0740E124543228A828B83EF
:20512000E0B504CAA3E0B505C5A3E0B506C0A3E0B507BB22740A12455460012211BB124620
:205140003F740D1245547010740D124543905177124313785D74FFF2785BE22401F208E299
:205160003400F208E204F224FA7007F2905193124317740C0243344C697374206F662062B6
:20518000616420626C6F636B206E756D626572733A0A0D00740A124554600122785BE2FC55
:2051A000E4F208E2FDE4F2FE9051B112431302432A546F74616C206E756D626572206F6653
:2051C0002062616420626C6F636B73203D200090E900E0FAA3E0FB780479E988828983C3E5
:2051E000AD007C0489A0E2F5F0C0D0E82401F8500205A0D0D0E0A395F0DCEB4019A805EAA7
:20520000B582DCEBB583D8E82404F8500109B502CAE9B503C6227C04E824FFF8400215A09A
:20522000E58224FFF58240021583E0F5F0E2F0E5F0F2DCE480A1740E12455470012274011F
:205240001245491245A731CF740D1245439052B01243131246DD905193124317785B7A0237
:2052600012E194E5FFF27A047BE9785EEA2404F208EB3400F28A828B8379047A0412E1B73D
:20528000313E785EE2FA08E2FB90E900E0B502DAA3E0B503D5740E124549785BE2FC08E251
:2052A000FD85398375829CE02CF0A3E03DF0219453756D6D617279206F6620626164206210
:2052C0006C6F636B206E756D62657273206F6E20647269766520008539A078A2796E7A04D5
:2052E00012E19A12463F1245AD7428752B021229BB122D3D1245A71231D3600420E2E42256
:2053000075A00078008539837582A67A0412E18C75A0E0E4221245AD7400124543122735AA
:205320006008740012454902496774001245492290537D1243130512E480218510838511F7
:2053400082E0A3858310858211FC740412432ED51427E512B4010122E5132410F513FC9082
:205360005193124317BC000512432D7C0012432D90540812431F751410D512BF222020207B
:20538000202020203020202031202020322020203320202034202020352020203620202088
:2053A0003720202038202020392020204120202042202020432020204420202045202020F6
:2053C000460D0A2020202D2D2D2D2D2D2D2D2D2D2D2D2D2D2D2D2D2D2D2D2D2D2D2D2D2D7E
:2053E0002D2D2D2D2D2D2D2D2D2D2D2D2D2D2D2D2D2D2D2D2D2D2D2D2D2D2D2D2D2D2D2D0D
:205400002D2D2D2D2D2D2D00207C0090544012431390E04E7410F075120490FE00E054703A
:20542000B4700F758207E0B47900400274782408F5127510FE7511007130784E740AF222CB
:205440005363736920726571756573742073656E7365207374617475732062797465732028
:20546000696E204865780030240E202A0B302F08E57C20E10302495F7834D0E0F218D0E0CD
:20548000F2E57C90548B75F003A4730254A6025BD4025BD474091245431245A77833E2C00B
:2054A000E008E2C0E0227404120062302903025A73C2101245AD753A0375A00012E1C912DE
:2054C00028BE122D3D122B94600D20E2ECD53AE912497F910B80C21245A775A00078088576
:2054E00039837582C17A1C12E18C7810903B46123B317003025785C22DD22C7804E27002FE
:20550000C22C1245AD753A037900202C03302D02797F123DDD1228E2122D3D122B946017BC
:2055200020E2E5D53AE2102C0A102DD6124983910B8199D22D80CB1245A78539A078C9902F
:205540003B3D123B31700675A0000257658539A078C9903B4F123B3175A0007003025736BE
:20556000780090E9007A0012E18C8539837582BFE0B40421D20590BF637403F03017FD124B
:20558000079512367E758278E07582B4F0758279E07582B6F0202C65202D6275A00012E16A
:2055A000C978037411F27582B6780CE0F27582BE08E060027401F97582B4E02342017582D8
:2055C000ACE0C449F27582AA08E0F27582BFE07A02B402010AB404070582E0B402010A7596
:2055E00082B7E02AFAA308E03400F208EAF27582B9087A0412E1847546150259FD1245AD00
:20560000753A0379BF1228E2122D3D122B94600820E2F0D53AEDA12C1245A775A0007AFF88
:20562000123DF6303005C2100257F6C21175460075A0E97A03123DF6705EA90075A0007A4B
:2056400003123DF670527B027C017D00C210125A997B048539837582B4E0FCF549125A9968
:205660007B067C00125A997B087582ACE0F547F5F07582B6E0F548A4FCADF0125A997B0A70
:205680007582AAE02549FC7D00125A997B0C7C007D02125A99125A7E8539837582BFE064F1
:2056A00004606475A0E97A04123DF6705AA90075A0007A04123DF6704E7B03E5482403FC8A
:2056C0007582B7E02CFC0582E03400FD125A997B05AC477D00D210125A997B077582B9E08E
:2056E000FD0582E0FC125A997B0A7582BBE0FD0582E0FC125A997B0C7582BDE0FD0582E04A
:20570000FC125A99125A7EE5467003025A1E75A000E4F8F27802F208E2600B7809E4F20883
:205720007402F208E4F208AA46E82546F54690010012E184804C12E1C978017403F27803B0
:205740007408F2780A7402F2780C7403F2087416F27823742AF208740BF208E4F275463211
:20576000D2120259FD12E1C978047420F208740AF2087402F2780B741EF2780D7401F275DF
:2057800046100259FD8539A0787D79727A0412E19A786E7A0412E1947546FF753A038546F0
:2057A0002B742A1229BB122D3D122B9A600920E2EDD53AEA025A678539A0786E7A04790484
:2057C00012E1A1E54603FB123E447804796E7A0412E1A8787279047A0412E1A1123E547867
:2057E0000479727A0412E1A8ED4E4F70AE754602BC00A8025A73753A0375A00012E1C9790D
:20580000BF853983758285E004F5A0F012E1C91228E2122D3D122B94600920E2DCD53AD94F
:2058200002552C753A03797F853983758285E004F5A0F012E1C91228E2122D3D122B946090
:2058400018C0E0853983758285E0C39402F0D0E020E2D3D53AD002552C758285E0C3F54867
:20586000F5A09401F5479401F0F583F8F9F582E3FB8547A0E4F0080582E2F0080582E4F07B
:20588000080582E2F0E27549046014F0FA2404F549E4058208F0DAFA15827402F00582E59F
:2058A00049F9F8E9B503004003025A1E758339758285E0F583E549F5828548A0E3543FFAC9
:2058C000894D09E370030980DAF54A8547A0C003123DF6884CD0036003025933E2F0B4035C
:2058E000061259B302590CB42022C000C083C0828539A078C9903B58123B3170068547A0C0
:205900001259E9D082D083D0008547A008E270030259330582F0080582FA2402F5F0E5492E
:2059200025F0F54612E18CC00312599ED003600312593CE54A2402254DF901A3A84CA94DA1
:20594000758339758285E0F5838549828547A0E2543FF008090582E2F5F08548A0E3B5F0CD
:2059600000501AC082ACF0C0E02402F5F0E54925F0F546E4F00582DCFBD0E0D082FCF0088E
:205980000905828547A0E2F5F08548A0E355F0F008090582DCEDC00312599ED00322124546
:2059A000AD7B00E546F91228FE122D3D122B9420E2EF22C000C001E54C240AF88548A0E5D9
:2059C0004D240AF9E309600D8547A0E408F28548A0080259D7080809E38547A060067402C5
:2059E000F208E4F2D001D00022E54C2402F87401F208F208080808F2087408F222753A0308
:205A00001245AD7B00A9461228FE122D3D122B94600C20E2EBD53AE8905AC61243131245D4
:205A2000A7123DC8758277E075823CF030240910120D75823A7403F0758239E04418F07542
:205A400082387404F075A00012E1C975280212187C122D3D758260E060030254B1122B9420
:205A6000C205600F20E2E412498712540B12367E025499C21012367E1253150254991011E0
:205A8000012275A00075830185468208E22402FAE5462AF5461802E18CEB28F8EB29F975DA
:205AA000A0E9E3700810101609E319601175A000201003EDF208ECF2D21110100118C3E882
:205AC0009BF8E99BF922466F726D6174207573696E672064726976652773206465666175EC
:205AE0006C7420706172616D6574657273007404657E120073753A027561008539A07872C3
:205B000079047A0412E1A17B5F123E545007123E44AB047C00780479727A0412E1A8EB7A7D
:205B200000785AF2602523F51712463F1245AD85172BE5321229BB122D3D122B9A60172094
:205B4000E2E78539A0785AE2B401051245A7EA22F561740180C91228A2E5616091D5E0F0DA
:205B6000808C30E10512496F801E30E00512496B801630E305124973800E30E405124977CB
:205B8000800630E50912497B12540B740122E4221245AD740012454385398375826E8563DD
:205BA000A078307A0412E18412200F60071249637A018013752B02742A1229BB122D3D1270
:205BC00031D320E2EF7A00740012454912463F1245A7EA22785B7A0812E194740E124549A3
:205BE0001252D778357452F208745CF2740C1245437414124543025CAB1251947414124520
:205C000049E57CB40160785FE204F208E4F275F0067860E2A4242108F2745D340008F278B9
:205C200060E204F2FC905D4F12431312432D905D5812431F785FE2FC12432D803175A0E074
:205C40001251947860E2B404C518E2F97868E2B501B47414124554600774071245546003D4
:205C6000125315125236740C124549025499753200E4F9FA7BBF7C00EA700E7A0675A0E0F0
:205C80007861E2F58208E2F583E4938CA0F3A3091AB900E40CDBE1E532703B75322A740D9B
:205CA000124549905D391243178013E57CB4010B740D124549905D441243177532287409F4
:205CC0001245498539A0786E7A0412E194787D79727A0412E19A51EE7019740912455460A0
:205CE00002808BE532B428C37414124554600261F9813D12513471627010740712455470B4
:205D0000051228A280D0719060028152E532B42A028171741412455470BC7409124543803D
:205D2000B5234E23462378AAAAAAAAAAAA555555555555FFFFFFFFFFFF57726974696E6761
:205D40002E2E2E0052656164696E672E2E2E005061747465726E2000205061737320009010
:205D6000E05EF075A00078007C102411F208B800F905A0DCF52274101245439061521243AE
:205D80001312451040F5B4790A74101245491245E8800690617C1243131249DC124FB8749B
:205DA000101245547003124E7190E01BE0F42401540790BF3BF090E01CE00314540FC4449D
:205DC0000F90BF33F4F01246E770030245DF785C7A0412E19478357481F208745EF2740CBD
:205DE000124543124BD6605F1252D785398375828C7A10123DD6741012455470057582A22C
:205E0000803130300512495F80D97582AAE0FCE4FDFE7582ACE023FB123E1575827D8539C5
:205E2000A0789079047A04C3E097F2A30809DAF875827D8539A078947A047B08E09BF27B46
:205E40000008A3DAF7809C785DE2F904F27869E2600BB501089060D5124313806709AC014E
:205E600090607F12431312432D757C00757D061246E7700774011245438006D57C4CD57DA6
:205E8000491246E79060A0124313905193124317124BD66028E539C394E12564FC74031283
:205EA000432E798E8539A0E3FC740912432E09B990F2785FE2FC740912432E80CD74011260
:205EC000455460831248E50245DF75A0007800E2B15F90BF247401F075320B7400125F1CD7
:205EE00075A0E912E1C912E1C790BF247403F075320974E9125F1C75830075A0E9E4F58269
:205F0000F87A02E0F5F0E265F06008906109124313803508A3B800EBDAE9803490BF21F06D
:205F20001582E4F0F533753404F535F5367537027933D2AA120B722000FD20080122D0E04F
:205F4000D0E09060EF12431375A0E0785FE204F2753200124BD67002C16F302408202A057F
:205F600012495F80EBE57E64041200738539A0789879047A0412E1A17410124554601F7B86
:205F800008123E448539A0789012445F400512447C5021789079987A0412E19A801F0C7B78
:205FA00019123E158539A0789412447C5006E4FDFEFF80EA780479987A0312E1A8E532705D
:205FC0000575322A803FB4282F75A00078007C1090E05EE02411FBE2B5030A08B800F505CC
:205FE000A0DCF1E15090612C1243131246DD8539A0788FE204F2E15075322875A0FF7A106E
:2060000012E1C7DAFB8539A07898796E7A0412E19A78727408F2087A0312E194125AEE6073
:206020009C125B62703B906064124313740912454385398375828EE004F0B4FF077401129C
:206040004543800312463F85398375826E79047A0412E1B712432A74071245546003125BDE
:2060600090025F50456363206572726F7220617420626C6F636B206E756D6265722000524F
:20608000756E6E696E672072656C696162696C6974792070617373206E756D626572200017
:2060A000546F74616C206E756D626572206572726F72733A0D0A4472697665202020204566
:2060C0006363202020202044617461202020202020446D6100436F6D706C6574696F6E20D4
:2060E0006F662072656C696162696C69747900446D61206572726F7220647572696E6720EC
:20610000646D612074657374004461746120636F6D70617265206572726F722064757269CE
:206120006E6720646D6120746573740044617461206572726F7220647572696E67206469FE
:20614000736B2074657374206F6E20647269766520004163636573732055534552204152C6
:206160004541206F66206469736B205B59206F72204E2C6465663D4E5D3F20004578657260
:20618000636973696E6720646961676E6F737469632061726561206F6E6C79001245E874EF
:2061A000111245431249DC302409202A0612495F0245DF1252D78539837582B4E020260B18
:2061C000700990625E1243130245DF740712454375827D79047A0412E1B77B01123E5478A2
:2061E0005C1246B478531246B490622912431312448A740B12455470061253150245E37445
:206200000612455470E38539A0796E78047A0412E1A890627812431375A0E0785C12447C33
:2062200040C7125B9070D280C0456E74657220626C6F636B206E756D62657220746F207271
:2062400065706C616365202872657475726E206B657920746F2065786974293A20004E6F66
:2062600020737061726520736563746F7273206F6E20647269766500496E6974696174694E
:206280006E67207265706C6163656D656E74001245E874111245431249DC30300612495FC4
:2062A0000245DF30240D1252D770089063101243138018124C099062D11243131246DD12C8
:2062C000531512463F9062EE1243171246DD0245DF5374617274696E67207263742077725A
:2062E000697465206F6E2064726976652000436F6D706C6574696F6E206F6620726374206D
:206300007772697465206F6E206472697665200052637420616C72656164792077726974EA
:2063200074656E206F6E206472697665200074111245431249DC203006202A03202406126A
:20634000495F0245DF1252D7600F741312455470089063A712431380E975460075470085B4
:2063600039A078B5E2F5F078B2E2A4FB78A279047A0412E1A1123E447804796E7A0412E194
:20638000A879AAE3FB123E65E5F0700122EBC395F0FB786E79047A0412E1A1123E44780484
:2063A000796E7A0402E1A84572726F722072656164696E672052637400AC46AD477E007FBD
:2063C0000002432A85398375826E7A04C3780220220118E038F07800DAF9E5462401F546B4
:2063E000E5473400F547227B108539A0786E79047A0412E1A178047A0412E1AF7A1C7404D7
:2064000078008013BB08097B01123E447B0880E57A20C374017800F0C833A3DAFA7A20D394
:2064200074FE78FFF0C833A3DAFADBD8227413124543712E12463F752B0274281229BB129F
:206440002D3D122B9A602220E2EABC080B90650D12431371B90245DFC0E09064D812431330
:2064600071B9D0E0125B62802D90E90071E790E90075A00078007A023022027A04E0FBE2E4
:206480006B600A9064AC12431371B9800908A3B800EB05A0DAE771C4809A4572726F72203F
:2064A00072656164696E67205263740044617461206D6973636F6D70617265206174206476
:2064C0006961676E6F7374696320626C6F636B206E756D62657220005374617475732065FE
:2064E00072726F7220647572696E672072656164206F6620646961676E6F737469632062B6
:206500006C6F636B206E756D6265722000436F6D706C6574696F6E206F6620726561642C12
:20652000206E756D626572206F6620626C6F636B732072656164203D200074131245437154
:206540002E9065B212431312463F752B0274281229BB122D3D122B9A20E2EC701571C480B8
:20656000E6C0E090661012431371B9D0E0125B6280EBBC08EC9065D112431371B99000007B
:2065800071E712463F752B02742A1229BB122D3D122B9A20E2EC70099065FC12431302457C
:2065A000DFC0E090663E12431371B9D0E0125B6280EC536561726368696E6720666F722090
:2065C0006120626C616E6B20626C6F636B2E2E2E005374617274696E6720777269746520C6
:2065E0006F6620646961676E6F7374696320626C6F636B206E756D6265722000436F6D70FE
:206600006C6574696F6E206F66207772697465004572726F7220647572696E6720726561A4
:2066200064206F6620646961676E6F7374696320626C6F636B206E756D6265722000457211
:20664000726F7220647572696E67207772697465206F6620646961676E6F73746963206237
:206660006C6F636B206E756D626572200074111245431249DC784E7410F2753A0375A0004F
:2066800012E1C91228BE122D3D122B94600F20E2ECD53AE99068671243130245DFC22DD2F6
:2066A0002C75A0007804E27002C22C1245AD753A037900202C03302D02793F123DDD1228E0
:2066C000E2122D3D122B94601920E2E5D53AE2102C0C102DD69068671243130245DFD22DF3
:2066E00080C91245A7202C19202D1675A0007800E2F549F547E4F2F548F54A1267960245FA
:20670000E3753A00753BFF75A0007800E204F5497803E20428F8E2543FF2B53A004002F579
:206720003AB53B005002F53B08E22804F8B5490040E4AC3BAD3A7E801246CA9068A01243A2
:2067400013AC3B12432D90686512431FAC3A12432D907CC412431F12448A740B12455470C6
:20676000030245DF740612455470C775A000AA04123DF6600890683112431380B588480886
:20678000E22402F54775A000E4F8F27802F2754A01126796C17A7510008548118547121209
:2067A00053307C00AD471D1246CA906840124313AC471C12432D907CC412431F12448A74DE
:2067C0000B1245546033740612455470D58C4B7C007DFF1246CA90688112431312448A74E0
:2067E0000B12455460BC740612455470E275A000E54B2548F8ECF280A99068D0124313125D
:20680000451040F5B47927753A031245ADAB4AA9491228FE122D3D122B94601220E2EBD544
:206820003AE890690312431312540B0245DF0245A750616765206E6F7420666F756E640023
:20684000456E7465722062797465206E756D62657220746F206368616E676520696E2068B5
:206860006578205B302D004D6F64652073656E736520636F6D6D616E64206661696C65641C
:2068800000456E746572206E6577206461746120696E20686578205B302D46465D3A20005F
:2068A000456E7465722070616765206E756D62657220696E20686578202872657475726E30
:2068C000206B657920746F206578697429205B00446F20796F752077616E7420746F206938
:2068E00073737565204D6F64652053656C656374205B59206F72204E2C206465663D4E5D0D
:206900003F20004D6F64652073656C65637420636F6D6D616E64206661696C656400496EB8
:20692000717569727920636F6D6D616E64206661696C656400906C251243131245BF905119
:206940009312431790BF637403F03017FD12079575460875A0E112E1C97539E1154690BF7F
:2069600068E546F090E01EF090BF64F015827401F07A061582E4F0DAFDF5291582F0158279
:206980007406F0752A017544FFD20390BF637444F07441F0E4781579167A05300311D8FBCB
:2069A000D9F9DAF7F000E060067403F0026B653048AA855958F5477539E17548008539A087
:2069C00012E1C97803E54DF278067406F278BF7404F278857400F2788AE547F208E548F227
:2069E00044C07837F2E548C4237839F275240074017832F2F525753A031245AD122938123C
:206A00002D3D1231D330E308E545B40603026A6B122926781579167A05300323D8FBD9F926
:206A2000DAF720503890BF637403F03017FD787E79847A1ED8FED9FCDAFA12079580121224
:206A40002D3D122B94602720E41E20E2AC5403600CC228853983758232E054FEF090BF63B9
:206A6000E4F000E0600221A9D53A8E026B4CD2051245AD85398312367E1245A7600A8539D8
:206A800083758238E0B425E3906BFD12431FAC4712432D906C0D12431FAC4812432D853916
:206AA000837582C1E06037906C1312431F8539837582C17A08126BF5906C1312431F853973
:206AC000837582C97A10126BF5906C1612431F8539837582D97A04126BF5E41242B675820B
:206AE00087E07007758232E054FEF075827D7A04790412E1B77582AAE03024183022110301
:206B0000F07B02123E6575827D7A04780412E1AF7403802AFB123E657582ACE0FB123E653F
:206B20007582B77A02780412E1AF78007A067582B9E042000582DAF97401B80001047582C0
:206B4000BFD2E4F00539E53964EA60192048090548E54820E30221BD0547E54720E30665F9
:206B60004660F521BA1245A7C20575A00012E1C97800741FF208E57BA2E0740130B5045074
:206B8000027408F2087404F208E546F27B007539E00BEB75F019A4F80539E53964EA601EAD
:206BA0008539837582BFE030E404D202C2E4B40403C202E4300202D2E4F2C2E47001229064
:206BC0003D4623F993C90493F5828983E49370063002BEC202A3A3E493C210B48C02D2104C
:206BE000A3A983AA82853983F582E00830100123F28A8280D5E01242B6A3DAF9220D0A5357
:206C000043534920414444524553532000204C554E20002C20002C20524556204C4556454F
:206C20004C203D2000414C4C2044455649434553204D55535420424520504F574552454449
:206C400020555020414E4420524541445900740412454975A00112E1C912E1F0123B97F541
:206C6000F0E265F0600B7404124543906C7212431322556E70726F6772616D6D6564206FF8
:206C80007220636F7272757074206E6F7672616D00914E75A00012E1C975390275A00178B2
:206CA00000E208FC7B087E009002007A19123DD6903C0C123C8C7900E3B41F05903C8380EE
:206CC0001C30E402D2105407700122903C0223F993C904932402F582E93400F583123C8CC9
:206CE000758300850682A90078007A1912E18CAE82A80180B375A000E375A0E02275A0002C
:206D0000F380F67A0480067A0280027A01AB01780475A00012E1A8A90380DE7A0480027A31
:206D20000278531246B4AB0175A000A8017904C00212E1A1A90375A0E078571246B4126D42
:206D400056D00280C891F5300202C2E4FE1246CAAC06E4FDFEFF200535C083C0821243136C
:206D6000907CC812431F12432A907CC412431F12448AD082D083740612455470DC300204DC
:206D8000ECD2E4FC808585D05B740A124543785DE22402FA7B02C083C082E493A3B40A02D5
:206DA0000A0B70F6EA94104005AA031245BF785DEAF2D082D083124313907CBF12431F7451
:206DC0000A1245546011740A124549855BD0744E500274590242B212432A7857C00179045C
:206DE0007A04E2F70809DAFAD00181F585D05B5018C083C082124313906E3612431F12450C
:206E000010D082D08340EA8016C083C082124313906E2C12431F124510D082D08340EA70CC
:206E200004855BD022B47902D322C3222C6465663D4E5D3F20002C6465663D595D3F200024
:206E4000D2059191200524907C1F12431312451040F5B47904D204800E9076A2124313120A
:206E6000451040F5B479043135D214755C007900741F91FD092004097C017D08907A31B17C
:206E8000450920040C7C027D20907A44B14520E0F40991F5F546540791FD300406AC46B191
:206EA0000B80097C007D07907A6CB1455346F84246907A8BE546A2E4300504B186800F2054
:206EC0000402B1ECE546300401C392E4F546907AAFE546A2E7300504B186800F200402B1F8
:206EE000ECE546300401C392E791FD097C007D0F907911B145E409F309B919FB74151245C5
:206F000049741612454930050791F570030245DFD20230040C91F5C2E4F5467C14B10B805C
:206F20000D7C017D0490752FB145C2E4F546C2020991F5F5240991F5F525E9F551E546B418
:206F40000109E9754B142414F98026B4031C200410907C6CA22F300504B1868004B1EC9220
:206F60002FE9754B082408F98007E9754B0E240EF991F5F5260991F5200408202F05127D64
:206F8000F091F5F527E5463004077404F546754B0EC210B4041DD210301418E551254BF9F4
:206FA0001974E1255CF58375828BE091FD191582E091FDE551F9200429202F12907C51A280
:206FC00030300504B186801AB1EC923050145324DF202A0E30240B302F05D2305324FB537C
:206FE000243FE5466403600302706B532445D224A222E492E091FD30040F7C00202A0520D4
:207000002F027C01126D0B8011302F047C0080F47C007D019079B7126D45A2E09222092077
:207020002F207C017DFF9079E7126D45097CC8E4FDFEFF1246B274FFFCFDFEFF907A091291
:207040006D1B740329F9302F0C09907C8C124313C22A02741B907B93A22A300506126D8674
:2070600002729D126DEC922A02729D2004283010295324E953257BE924053024022406F934
:207080002024E5126CF56007E92402F90271D9E92402F902729D190274AF20051130140EBA
:2070A00090766012431312451040F5B479C9E92405F9126CF5F5F0E924FCF9126CF5F54C57
:2070C00025F0F54D126CFD7C017DFF90757E126D45F547B54D0280057415124543097C0130
:2070E0007D3F90760F126CF5F54D126D45F548B54D02800574151245437B00E546B4010200
:207100007B02B402027B03C003E92404F9126CF52BFBE924FDF9126CF585034D2B126CFD65
:20712000F54E09126CF53400126CFDF54F197C14E4FDFEFF1246B27CFF7D0F907634126D4C
:207140001FECB54E06EDB54F0280057415124543C004C005AB4D123E548C4E8D4FD005D000
:2071600004D003123E548C498D4A126D0709097C007D03907CCE126CF5F5503030077400E7
:20718000126CFD8003126D45F5F0B550028009C0F07416124543D0F0E924FCF9E547C3959E
:2071A000F0F547126CFDE92405F9E5F0700A126CFD5324DF090271D97C027DFA907D5A123A
:2071C0006D45FBAC49AD4A123E548C498D4AE924FDF9126D07E92404F93005062030202068
:2071E000261D20301D907AD7A225300506126D860272DA126DEC9225500853243F800302F4
:20720000729D2005FA2024F7741512455470F0203007741612455460E6E924FEF9741612FF
:2072200045546006E924FEF98030126CF5606CF5F0E4126CFDE924FCF9126CF5F54C25F04D
:20724000126CFDE92405F9E4126CFDE924FEF9126CF5F54F19126CF5F54EE4FDFEFFAC4CE9
:207260007B02C001123E65D001F54DAC4EAD4FAB4C123E15E924FEF9126CF5FBC001123E33
:2072800065D001E5F0C36006E54DB5F000E43C0909126CFD09E43D126CFD09090920253AF7
:2072A000302403302A34907B07A226300508126D86302626800B126DEC92264004C22780F6
:2072C00019200410907B3EA227300505126D868009126DEC300401C3922730240302741B83
:2072E00020101190770D30051CA221126D862021240273CAC22175A000A8017A0412E194D6
:2073000075A0E080EC7407B55C0280E8A221126DEC50E1D221300511785DE22405F0B410EA
:207320000040067405F01245BF907734124313C375A000E99406F9E3F54709E3F54809E35D
:20734000F54909E3F54A09090975A0E0740A8548F0A4FCADF0E4FEFFAB47123E151246B2FA
:2073600012432A907B9112431FAC49AD4AE4FEFF7B0A123E54AB48123E15AB47123E157861
:20738000531246B412432AAB0175A000A801790412E1A1A90375A0E078571246B430050BD8
:2073A000907CBF12431F12432A801F907CC812431F12432A907CC412431F12448A740612F9
:2073C00045546003027329126D03740429F920104AE546B4012CE4FCFDFEFF1246B27CFF12
:2073E0007D0F9077D3126D1F09097CFF7D0F9077FA126D1F09097CFF7DFF9077BB126D1F68
:2074000009099077A3126CF5A2E0300505126D868009126DECE492E0126CFD9076ECA22003
:20742000300505126D868005126DEC9220907BEDA22E300505126D868005126DEC922E9024
:207440007B67A228300505126D868005126DEC9228907BBFA22B300505126D868005126DBD
:20746000EC922B0930141AE546B4041574E1255CF58375828AE0126CFD090582E0126CFDEF
:20748000197C007D07907821126D45097C007D0790783F126D4509E975F01984741995F0CC
:2074A000600975A000FAE4F309DAFCE924E8F9E524126CFD09E525126CFD89F0E9254BF9D3
:2074C000E526126CFD09E527126CFDA9F0E92417F9200527302102055C055C7408B55C02F0
:2074E000801C126CF5C36007D3300405026EFCC214C20490785D126DEC5003026EFCE412BA
:207500006CFD90788B12431312451040F5B47903026E6B9078C112431312451040F560F340
:20752000B47909123BB690BF637403F00245E35354353036203D203120202020455344493A
:207540002F454D424544444544203D2032202020204F70746963616C203D203320202020A7
:207560004175746F2D73697A65203D20340D0A5479706520636F6465205B312D34005068A0
:2075800079736963616C2067656F6D65747279206F6620646576696365206D6179206E6FF1
:2075A0007420626520616C74657261626C652E0D0A496E207468697320636173652064652B
:2075C000766963652064656661756C742077696C6C20626520757365642E0D0A0A546F74E9
:2075E000616C206E756D626572206F6620706879736963616C20736563746F72732070658B
:207600007220747261636B205B312D32353500546F74616C206E756D626572206F6620701C
:207620006879736963616C206865616473205B312D363300546F74616C206E756D62657249
:20764000206F6620706879736963616C2063796C696E64657273205B32302D3430393500EF
:20766000446F20796F752077616E7420746F206368616E67652064726976652773207068AB
:2076800079736963616C2067656F6D65747279205B59206F72204E2C206465663D4E5D3FF4
:2076A0002000446F20796F752077616E7420746F206175746F2D636F6E66696775726520B5
:2076C000686F7374206164617074657220616E64207363736920627573205B59206F722067
:2076E0004E2C206465663D4E5D3F200044697361626C65207363736920646973636F6E6EE6
:2077000065637473205B59206F72204E00446F20796F752077616E7420746F2073706C6992
:207720007420746865206472697665205B59206F72204E005374617274696E6720626C6F4E
:20774000636B206E756D62657220666F7220326E64206C6F676963616C2064726976650DE5
:207760000A77696C6C206265207472756E636174656420746F20747261636B20626F756E6A
:207780006472790D0A456E746572207374617274696E6720626C6F636B206E756D62657225
:2077A000205B0052656D6F7661626C65206D65646961205B59206F72204E00537465702092
:2077C000726174652F636F6465205B302D363535333500526564756365642077726974654C
:2077E0002063757272656E742063796C696E646572205B302D343039350057726974652017
:20780000707265636F6D70656E736174696F6E2063796C696E646572205B302D34303935ED
:20782000005363736920636F6E74726F6C6C6572206164647265737320205B302D370053CA
:20784000637369206C6F676963616C20756E6974206E756D626572205B302D3700446F2083
:20786000796F752077616E7420746F20636F6E66696775726520616E6F7468657220756ED8
:207880006974205B59206F72204E00446F20796F752077616E7420746F206368616E676535
:2078A00020616E7920706172616D6574657273205B59206F72204E2C6465663D4E5D3F2027
:2078C00000202A2A20414C4C2044415441204F4E2044524956452043414E204245204C4F56
:2078E0005354202A2A0D0A444F20594F552057414E5420544F204C4F414420544845204EDA
:207900004F5652414D205B59206F72204E5D3F2000556E6974206F6666736574206966208D
:20792000616C7465726E61746520636F6E74726F6C6C657220616464726573732069732001
:2079400073656C65637465642C206F720D0A756E6974206E756D62657220746F20617574C4
:207960006F626F6F742066726F6D206966206E6F7420616C7465726E61746520636F6E74FC
:20798000726F6C6C65722E0D0A456E74657220756E6974206F66667365742F6175746F2D78
:2079A000626F6F7420756E6974206E756D626572205B302D31350030203D203531322020C7
:2079C00062797465730D0A31203D20313032342062797465730D0A426C6F636B2073697A35
:2079E00065205B302D31004E756D626572206F6620626C6F636B73207065722074726163EC
:207A00006B205B312D3235350053697A65206F6620647269766520696E20626C6F636B7327
:207A2000205B3230302D3432393439363732393500446D61207468726573686F6C64205B79
:207A4000312D3800446D612062757273742064656C617920696E206D756C7469706C657309
:207A6000206F662032205B322D333200486F7374206164617074657220736373692061642A
:207A80006472657373205B302D3700456E61626C65207363736920706172697479206368F9
:207AA00065636B696E67205B59206F72204E00456E61626C6520455350206368697020736C
:207AC0006C6F77206361626C65206D6F6465205B59206F72204E00446F20796F752077610D
:207AE0006E7420746F20656E61626C65204D534350207265706C6163656D656E7473205B29
:207B000059206F72204E00446F20796F752077616E7420746F20656E61626C6520747261A2
:207B20006E73706172656E74207265706C6163656D656E7473205B59206F72204E00446FC1
:207B400020796F752077616E7420746F2069676E6F726520464354206572726F7273205BF2
:207B600059206F72204E00456E61626C652073796E6368726F6E6F757320646174612074BD
:207B800072616E7366657273205B59206F72204E002D00446F657320646576696365207363
:207BA0007570706F7274206D756C7469706C6520777269746573205B59206F72204E00444A
:207BC000697361626C6520686F73742061646170746F7220706F6C6C696E67206F662064BE
:207BE00072697665205B59206F72204E0050726576656E74206D616E75616C207370696E30
:207C00002D646F776E206F66206D6F756E746564206D65646961205B59206F72204E0045C6
:207C20006D756C6578206175746F6D61746963207365742D7570206F662055437878205B9C
:207C400059206F72204E2C206465663D4E5D3F200046756C6C206361706163697479206D0C
:207C60006F6465205B59206F72204E004973207468697320612043442F524F4D2064657651
:207C8000696365205B59206F72204E004E6F20757365722073657461626C65207061726110
:207CA0006D65746572732C207573696E672043442F524F4D2064656661756C74732E005DFB
:207CC000203D20005D3A20002C6465663D004E756D626572206F6620737061726520736547
:207CE00063746F7273206D6179206E6F7420626520616C74657261626C65206F6E206465E8
:207D0000766963652E0D0A496E207468697320636173652064657669636520646566617577
:207D20006C742077696C6C20626520757365642E0D0A0A4E756D626572206F6620737061C2
:207D4000726520736563746F72732070657220747261636B205B302D33004E756D62657219
:207D6000206F6620616C7465726E6174652063796C696E64657273206D6179206E6F742049
:207D8000626520616C74657261626C65206F6E206465766963652E0D0A496E2074686973EF
:207DA0002063617365206465766963652064656661756C742077696C6C2062652075736546
:207DC000642E0D0A0A4E756D626572206F6620616C7465726E6174652F73706172652063E5
:207DE000796C696E64657273205B322D32353000907DF875F003A473027E0A027E13027E87
:207E00001C027E25027E2E027E37907F39124313027E40907F53124313027E40907F6D12B4
:207E20004313027E40907F87124313027E40907FA1124313027E40907FBB124313027E40A4
:207E4000C001200518907E6012431312451040F0B4790A7C007D05907E93126D45D001222A
:207E6000446F20796F752077616E7420746F206368616E6765206D65646961204944205B27
:207E800059206F72204E2C20646566203D204E5D3F2000506C656173652073656C6563741E
:207EA0002061206D65646961204944206E756D6265722066726F6D207468697320746162C8
:207EC0006C65202D205B302D355D0D0A6F7220747970652052455455524E20746F20757335
:207EE000652063757272656E742064656661756C740D0A0A30203D20524138310D0A3120C3
:207F00003D20524138320D0A32203D20524139300D0A33203D20524139310D0A34203D20B9
:207F2000524139320D0A35203D20524435340D0A4D656469612049440043757272656E74F4
:207F4000206D656469612049442069733A20524138310043757272656E74206D65646961FF
:207F60002049442069733A20524138320043757272656E74206D6564696120494420697355
:207F80003A20524139300043757272656E74206D656469612049442069733A205241393188
:207FA0000043757272656E74206D656469612049442069733A2052413932004375727265BC
:207FC0006E74206D656469612049442069733A205244353400F4557E8005457E8001F49089
:207FE000BF80F57ED2E6D2E5F022C082C08390E47FC0E0E07002748004F0F582D0E0F0D015
:2080000083D08222C0D0C082C083D2D3FE90BF31E030E1087402F0D20202808590BF30E098
:2080200020E0FC0582E030E102D202F52A54F3F0300052305730303E1EE57F543F20B5020D
:2080400054036008157FE57FF590801A757F3F20B5F4757F0380EF057FE57FF59054C02047
:20806000B50254FC701B20541620551520501430570890BF30E532F0800B3051068006D257
:2080800009D208C200EED083D082D0D032C0D0C082C08343D018FF90BF64E0F52990BF6532
:2080A000E030E73B90BF637402F07400F0C22F7C4974E42CF583758236E4F00582F0058261
:2080C000F0DCEE90BF67F07A0279FF78FFD8FED9FADAF612A858D227D20AC2360281852055
:2080E0004D03304E23D20FD224D20A756606C22F854183758236E4F00582F00582F090BF83
:2081000067F090BF63741AF030E20030E40EC220E529540775F003A490818D7330E53420D3
:208120002423102220102122302040D20BD20AC220C22F854183758236E4F00582F00582EF
:20814000F090BF67F0D22702818590BF637444F002818530E31230E20302834C30250302C1
:2081600082D830232002838430E61AD224D20AD227C22F854183758236E4F00582F00582F5
:20818000F090BF67F0EFD083D082D0D0320281FB0281A502825E02828002850F02850F0229
:2081A00082E8028330300E0D75660690BF63741AF0C20ED224D226D22890BF147407F0E5D9
:2081C0003C253AF53AE53D353BF53BB4DE005027302D08753C80753D008006753C00753DD9
:2081E0000490BF60E53CF00582E53DF090BF637400F07490F0808ED22E808A300E0D7566DA
:208200000690BF63741AF0C20ED224D226C22890BF147405F0E53C2560F56090BF10F00565
:2082200082E53D3561F561F0241C5003F561F0C3E53A953CF53AE53B953DF53B853A3CE501
:208240003A853B3D453B70993024AC90BF60E4F00582F090BF637400F07498F0218590BF5D
:20826000637401F078447A068541838882E090BF62F008DAF390BF637400F07410F0218521
:20828000302648C22690BF60E0FA0582E0FB302816C3E53C9AFAE53D9BFBEA253AF53AEB6C
:2082A000353BF53B0282CB90BF63E4F090BF67E0541F2AFA50010BC3E53C9AFAE53D9BFB90
:2082C000C3E53A9AF53AE53B9BF53B90BF637401F07411F0D2252185C22590BF62E08541A1
:2082E0008375824AF002838490BF637401F090BF62E566F0B4012C854183758240E090BF2E
:2083000062F0854183758241E090BF62F0854183758242E090BF62F0854183758243E09013
:20832000BF62F090BF637400F07410F0C226218590BF63E4F090BF67E0541FFE90BF637461
:2083400001F07400F07410F0D223218590BF62E0F890837CE54693FB90837CE548935860E1
:2083600003C868F8E8B5180790BF62E020E705D23602839D5407B547F60284550102040818
:2083800010204080C22390BF62E0202F0D20E70D20242E7034D2220283C1028473D224E5E3
:2083A00066756606B40114C22F854183758236E4F00582F00582F090BF67F090BF63741A9E
:2083C000F090BF637412F02185B40404D22180F1B40724E566B401C58541837582377434FC
:2083E000F074050582F090BF67E4F0854183758236F075660880CAB402583026C4C22690E0
:20840000BF60E0FA0582E0FB302816C3E53C9AFAE53D9BFBEA253AF53AEB353BF53B0284DA
:208420004BEE2AFA50010BC3E53C9AFAE53D9BFBEA2560F560EB3561F561241C5002F561D0
:20844000C3E53A9AF53AE53B9BF53BE4F53CF53D61C1B4030261C1B40117305C148541838D
:2084600075823AF0854183758239743AF0D22F61C1619DFB854183758239E004F0FAF582EA
:20848000EBF0BA3E6AC22F85418375823BE0B403600582E0B4015A0582E0B43400500774AC
:2084A00034FA7C05801975F004A4FCE4FEFDE5F060010D7B2A12C5E7E0FAE5F060010C05C5
:2084C00082E0B410004002740FFE90BF67F0854183758236F00582EAF00582ECF090BF662E
:2084E000F08541837582397439F0E566B4010461C1619D85418375823F7401F0A37403F064
:20850000A37401F0A3EAF0A3EEF075660161BBD224D20FD20AD2272185D51620751680C035
:20852000D0C082C083D2D3FF90E402E0601FFA758203E0C39A400E7409028D7BD5300575E8
:20854000301A053132E55A7004E02405F0AC4974E42CF583758203E0700A75822FE0601AF8
:2085600014F08016F58375820AE0600E7582087B03D3E09400F00582DBF8DCD3EFD083D0CB
:2085800082D0D032BE50B841B842B843B849B84AB84BB851B852B853B854B855B856B85731
:2085A000B858B859E4F208F208F2089085B37A0502E1BF000000050190BF00E4F0F57F90B2
:2085C000BF327402F0740220B5027406F090BF80E0F4540F23FE90858493CE049390BF3650
:2085E000F00582EEF0857D7C90BF81E020E50F757C0090BF637402F07400F07403F090BFC1
:208600003474C0F090BF35740B20B5027409F090BF3374CFF0757D007581667590BD75B0D1
:20862000FF12E6A6C21D758901758800759800D2B875A88290BF80E07B0020E70312E8E07E
:2086400012897890BF35E020E733BB00F3B430F01582E0B403EAE4F005827401F0128978FC
:2086600090BF35E01582B444067541E502E2DAB446CE7407127FDA7541E502A9A530E60AEF
:208680001582E0F00582E0F080F612E8E07541E590BF35E0FF12895F90E40AF0A3F0EF23C1
:2086A000C412895F90E40CF0A3F090BF34E090E411F0D21810E702C2187004C218C21990AB
:2086C000BF3AF0E57D60057D88028D8590BF34EFF07D9005827410F030180790BF32E04473
:2086E00040F012897875A0E490BF35E0F5147805F21582E030E004D21954FEF51318F21276
:20870000A88A90E411E090BF34F005827420F030180790BF32E04440F012897812A9147DC1
:20872000A090BF34E0F51590E406F07B0090E40AE024FF23232513F510E5143BF511E5150F
:208740003BF512E5102404F54D90E407F0E5113BF54E0582F0E5123BF54F0582F090E40CB5
:20876000E024FF2323254DF54AE54E3BF54BE54F3BF54C90BF35E030E739E41582F00582FB
:20878000F0793C90BF31E020E20AD8F7D9F5757D15028D8590BF34E0FC0582E04C60030299
:2087A0008D8290BF31E020E10AD8F7D9F5757D15028D85F07906D375A000E4F8FAF233082D
:2087C000DAFB05A0D9F790BF20E4F005827400F090BF247401F0E513C32019049404800237
:2087E0009408F533E5149400F534E5159400F535793390E40CE0FF90E40AE02F50037537B0
:2088000004335003433702335002053754FC30190224042404F536753203D2AA128E5E2037
:2088200000FD300806757D07028D8575A00012E1C9790412E1C7D9FB90BF20E4F0058274D6
:2088400000F090BF247403F07532017933128E5E2000FD300806757D06028D8575A000AAD6
:2088600036AB3778000BBA00011B7480C333FCE26C6006757D06028D85EC0808D80205A066
:20888000DAEBDBE990BF20E4F005827404F090BF247401F07532037933128E5E2000FD30A4
:2088A0000806757D07028D8590BF32E04401F090BF347452F07DC005827440F03018079087
:2088C000BF32E04440F090BF31E030E2F990BF32E054FEF090BF34E0FF54FC60050324F90E
:2088E00050027407201F0530E3027407540F457B90BF33F4F090E415F0EF30E11EE57C60F6
:208900001A8551A090896912E1E178201285A4782AE57CF278517958128F0A90BF34E030D1
:20892000E0FCD28C90E411E06002D218D2A8D20412A85890BF81E030E561AC497541E51222
:208940008A9EB4081090BF80E030E61012A8467541E502899B0541DCE67541E502899B5470
:2089600007FA74800A23DAFD221D011E0A280729071018121013010090BF31E0F030E2F87F
:208980002290BF35E4F0C2AF80FE740290BF35F0317890BF34227401127FDA300209C20257
:2089A000D2037401127FD5101C1BE55560057855028C83E55760057857028C83E55960051F
:2089C0007859028C83E5536003028F8C300315E551700BE559600D78597950128F0A128A78
:2089E000BB2003EB3016053027B1C216201730854183758203E070233027A0E54924E50533
:208A000041B541037541E5854183758201E0700875822FE0601880830292FEF55BF5A0856B
:208A20004183758205E0C0E01582E0C0E0227539027401F0128A9E854183758206600E209A
:208A4000E30920E003D539EC7423F0219BE0543FB423497404F090E410E030E73FE551708F
:208A60000BE559603778597950128F0A8551A07A40781012E19478107420F27818E541C30B
:208A800094E5F2781C7440F278208541837582087A2812E18478517956128F0A219B12C562
:208AA000D2758244F0F521758234E0F5460582E0F54712A7B93027FD0295C77851794D12F5
:208AC0008DF820E71930190890E01DE090BF33F0C2033027082017057401027FDA2290BF20
:208AE000207410F00582E551F0F583753628128D583008057401028D7B855183758213E0F4
:208B0000146005740E028D7B758211F01582742CF0753802794D128DD2ED30E629E54DB538
:208B20004A07E54EB54B028017794A753205128E973008057406028D7B90BF39E030E7062C
:208B40007538FC128D9EE54DF54A2404F54DE54EF54B3400F54EE54FF54C3400F54F90E409
:208B60000DE014F070161582E00582F090E407E0F54D0582E0F54E0582E0F54F85518375D0
:208B80008212E054F024D050057414028D7B30E4F830E50122E55AB40E05740A028D7B056B
:208BA0005A90E403E4F085518375821CE0FB128ED87851600E758210F0EB54F8700E7952A3
:208BC000028F0A7A08D0E0D0E0028C4A7904E475820BF0158274FFD9F9758219E0700B1591
:208BE00082E0C304954940096007D0E0D0E0028C64E024E5F5A078007901E2F583758202A9
:208C0000E4F0E27004E551F2F3E58370097802E2FEE551F28008758200E0FEE551F0E583C1
:208C2000855183758201F01582E0CEF06009F5830582E551F08003E551F28E51BE00038E57
:208C400050228E83758201E4F022868375821C7480F0758210740CF075821E7401F005822B
:208C6000EAF08013868375821CE0D2E7F075821E7403F00582E4F075821DE4F07954128FB5
:208C80000A219B7913128DF820E70F30190890E01DE090BF33F0D21C219B90BF247401F023
:208CA00090BF207410F00582E6F08683B857028007B855180517155AC3E517940E4006F587
:208CC00017740E8003E4C517758212F0753203758210E02404F536128D583008057402022F
:208CE0008D7B7538027913128DD2ED30E629E513B51007E514B51102801779107532051231
:208D00008E973008057406028D7B90BF39E030E7067538FE128D9EE513F5102404F513E5EE
:208D200014F5113400F514E515F5123400F51590E40BE014F070161582E00582F090E4044E
:208D4000E0F5130582E0F5140582E0F5157950128F0A7910D9FE219B75820FE0C2E0C394DB
:208D600004F5331582E09400F5341582E0FC9400F5357933128E5E2000FD22F57D7D800208
:208D80008D85757D1375A89090BF34E57DF0FF0582EDF0740FBF0901E4127FDE80FE90E446
:208DA00004E0F5330582E0F5340582E0F53590BF387401F00582E4F07532077933128E97AE
:208DC000300804740780B430180790BF32E04440F02230190890E415E090BF33F090BF38AF
:208DE000ECF00582EDD2E6C2E7F0753207128E97200801227407808330190A90E415E090D8
:208E0000BF33440FF090BF247403F090BF20740CF00582E6F075360475370075320190BFB5
:208E20003BE04418F0D23E128E452000FDC23E90BF3BE054E7F0200808868375820CE0FD0B
:208E4000227406A17B5321FC90BF3CE72402F4F0058209E73400F4F009E73400800F5321B8
:208E6000FC90BF3CE7F0058209E7F009E7543F20B5025403F57FF59090BF3EE536F42401C2
:208E8000F00582E537F43400F090BF30E532301F022408D200F022E5385480600274FFF575
:208EA0007B90BF3CE72538F0058209E7357BF009E7357B543F20B5025403F57FF59090BFB8
:208EC0003E74FEF0058274FFF05321FC90BF30E532D200F02000FD2224D85002E42294D742
:208EE00083220010142C1C0000000C2C2C0C000000000000200000002000000000000000B1
:208F0000000020242400202000008683758200E0F6F5A06007E4F07801F2800318F6F075A2
:208F20008201E7F0F5A0A7836006E5837800F22209A78322301954855BA07827E2604CFB24
:208F400090BF38E4F00582EBF090E4047A03793312E1B77538FA7532077933D19730080464
:208F60007407A17B90BF317404F090BF32E04440F0757D0890BF31E030E2F9757D1590BFE2
:208F800034E070F00582E070EBF57D228553A0781CE24480F2908FA0C2E7C2AF75F003A47E
:208FA000D2AF73028FB702902F02908A02923F79547853F10A219BE408F2B81FFA79040842
:208FC0007A0412E1A17819E2700718E2B54900400280DCE624E5F583758201E0C210604846
:208FE000F5A0F55B79047814E267700E0908B908F7758203E0B55B1780057800E280DFE4D0
:20900000F0C2AFF52190BF30F0C200D20ED2AF855BA0781CE2D2E7F2E408B824FA781E74DA
:2090200002F22010031292937401127FDA8080E408F2B81FFA790408E2F709B908F9781991
:20904000E2703A18E2B549005033E224E5F583758202E0C2106026F5A0F55B79047814E2A5
:209060006770150908B908F778088553837582247A0412E18C028FAF7800E280D88553A0DE
:2090800078247A0412E194028FAF7819E2700718E2B549004013781EE230E0087818E4F2C4
:2090A00008F280067853028C64E224E5F5A085538375821DE4305B07D2E3305802D2E4F029
:2090C000058278067A1612E18C78267A0612E18C028FAF8541837822E25423FA75820AE088
:2090E00054DC4AF008E2A2E4781EE282E20582E092E4F0305A277834E2FA75822AE05A60F9
:209100001CB4040114F564D239753902129583600F20E3F520E006D539F21039EC02922CC6
:20912000203903029204900000E004FDB40E005003029204900004E06005B404004002D278
:209140003490000CE0543FF020340302920475A0007A0F123DF6704908E2B40E4408E23047
:20916000E63FE564B4031574C0F2087480F2E82404F87420F27403F56402918D7440F20875
:209180007480F2E82404F8E4F27402F564753902129523603120E3F520E03C20E103D539EB
:2091A000EF75A0007A10123DF6702F08E2B40E2AE8240DF8E564B4030574010291BFE4F2B4
:2091C000753902129523605520E3F520E00920E109D539EF0291DA02922C75A0007804D2C8
:2091E00012C239E564B4030574850291EF7414F2753902129523602520E3F520E02E20E142
:2092000003D539EFC212C239E5646020753902129523600920E3F520E012D539F2E5646020
:209220000BB403010485418375821CF085418375821EE07836E2F0C234C212855BA0227879
:2092400020E2600778537A0C028C4A781D7A0312E1947822E254F090E410F0F27825E260DE
:2092600006E4F2F418800218E290E402F074FFF278267407F2087407F290928212E1E102C5
:209280008FAF285529432A302B372C302D382E052F010078007901E3FBF5836005E2758241
:2092A00000F0E2FA6006C583758201F0E4F2E554F3855B547005855B558007F5A0E55BF21E
:2092C000F5A0854183758200E0B55B09EBF07005A3F0A3F022758202E0B55B02EAF075826C
:2092E00001E0B55BEFEB6002F022EAF022854183758204D0E0F00582D0E0F002899B75820B
:2093000001E0758203F0F5A0F55B75822DE0F52B7A06758230794212E1B7856539781FE2D1
:2093200030E003753901305E0820E5030295B8C25E781CE2FA781DE4F2532703EA24E040D8
:209340003F2410401A9093535407C2AF75F003A4D2AF730294820296410297A50297BC90EA
:20936000936BC2AF75F003A4D2AF730293A00293A00297FB0293A00293A00293A00297D177
:20938000C20590938EC2AF75F003A4D2AF73029CED029D3A02A1710293A002A5480298B8F6
:2093A000757D14028D8578347A0412E19478207A0412E19402941978347A0412E19478204D
:2093C0007A0412E194AF0179307A04784212E1A8305B0D781DE2D2E3305804D2E4D25EF234
:2093E000A90702944A793078427A0412E1A8305B18781DE2D2E3305804D2E4D25EF23058A6
:2094000008781F7404F2E48004781FE4F218F2029451E4781FF218E9F2793078427A04122A
:20942000E1A8305B2C781DE2D2E3305804D2E4D25EF2029451781FE4F218E9F261A6781E78
:209440007401F208E9F261A67900781FE4F218E9F2781CE24480F2854183758203E4F0C2DD
:209460001E51933017012285418375822DE52BF07A04758230784212E1AF7401127FDA0230
:20948000899B854183758206E0B42311854183758206E0781EF2058208E0F280B4303705EB
:2094A0007800129786128A9E601020E00920E3ED30E103D539E7740380D28541837582064A
:2094C0007404F0753902781EE230E43A12C5D2F521758244741BF012A7B93027FD1295C701
:2094E000601B20E3F220E0CE30E40DEB540F600DB4020280C1D539DF0298A9D25AC25B12CE
:209500009CE1C25D8148129B9E60F020E3F820E00B30E4E4EB540F60E2B402028098D539DF
:20952000E580D512C5D27582447415F0740C30390605827410F0ED758248F0900000E4F02A
:209540000582F074100582F005827408F00582E4201206203402E564F005827807E4F00595
:2095600082D8FB753A0C30390385053AE4F560F561F53B90BF10F00582F012A7BE3027FD5B
:209580000295C712C5D2758244741AF0740C303908758246743FF074FF758248F0E490BF65
:2095A00010F00582F012A7B93027FD0295C7781FEAF2187406F261A6781E7412F2E408F226
:2095C000205D02C25E61A612962C605A30E15712C5D27582447403F07582487420F0C03CE5
:2095E000C03DF53C753D0090BF10744BF00582E541F0E4F53AF53B75252012A7C43027FD12
:2096000012962CD03DD03C600330E11A85418375824BE05470601175824DE0FBB40605E46D
:20962000758238F07410FA227404FA22300A087401200B0274042285418375824AE0540A91
:2096400022128A9E600F20E00920E3F530E103D539EF029729D239753902B183600F20E30A
:20966000F920E0EED539F31039ED029729900002E0A2E785418375820BE092E5F0303922F2
:20968000900000E004FDB40E0050030296A290000CE0543FF00582E0042582F582E582B566
:2096A00005EF753902756400B123600F20E3F320E0A0D539F31039EA029729C2398541831A
:2096C000758206E07009781EF2087401F2807B129B9E600620E3F8029729D25AC25B12C5B4
:2096E000D2F5217582447405F0E490BF10F00582F012A7B93027FDB1C7600620E3E0029714
:209700001F8541A0900001E0600A782074FFF208F202971F05827821E0F2180582E0F28552
:209720005BA011D3790002972B7923303708E970057801129786855BA085418375820778BD
:209740001FE4F0F2E9181582F2F075820878207A1E12E184815112C5D27582447412F07563
:2097600082487424F09000007824E4F00582D8FB90BF147403F0E490BF10F00582F012A710
:20978000B93027FDA1C712C5D2758244741EF0758248E830E005740102979CE4F012A7B9C2
:2097A0003027FDA1C7854183758206E0700211D3758206781E7A2012E1848151854183753D
:2097C0008206E070028148781EF20582E008F28112854183758206E0600A7923E9F00582DE
:2097E000E4F0811275820BE030E4047A10A1AE30E5047A20A1AED210029850854183758221
:2098000006E060148541831017227582067923E9F00582E4F002941275820BE030E4057A72
:20982000100295AE30E51B7A200295AE85418375822DE52BF07A04758230784212E1AF0254
:209840008996781EE230E608D2171293E51292EDD25812C5D27419758244F0101006058217
:20986000E0D2E0F012A7B9D2161292ED1295C720E3F2602F20E08D30E42FEB30E605D25A87
:20988000129CE01017A6EB540F6018B407087A201017990295AEB405057911029412B4029F
:2098A0000801041017860293E510170A798B7C0012A6A5029412012C854183758206E0600B
:2098C000188541837582067923E9F00582E4F078207A0812E194029412795C7A0878201210
:2098E000E1A178207A0812E194C258781EE2F56430E602D21730E155129CE030170F793066
:209900007A04784212E1A81294481292ED129B9E7007C25BD25A02995F20E3F120E00B30C1
:20992000E410EB540F60EBB4020510170A8092D539DB10170201A985418375822DE52BF073
:209940007A04758230784212E1AF02899630170F79307A04784212E1A81294481292EDE5AF
:2099600064532284C23C30E304D215C25D30E204D210D21330E709201506D2118002C25DB3
:209980007B04785CE6700508DBFAD21420130C7B047860E6702708DBFAD21330141F1017F7
:2099A00096800C129AF030141430131110177330110885418375822EE4F00293E530150653
:2099C000305A03029A8920133590BF80E030E525753C01753D00E563456245617010E560C6
:2099E000B401063011030299F1B404004007205D1FD235801B753C00753D01F08012855CD8
:209A00003C855D3DE53C453D7006753CFF753DFF129BB4604BC23520E02620E41B10170200
:209A200001A985418375822DE52BF07A04758230784212E1AF028996EB540F601DB4020567
:209A40001017DF01C1B408047908803FB405081017D07911029412B403C3205A2C105907C4
:209A6000103504C25D21A3301005129B12800C153CE53CB4FF02153D129AF0129B3A70209E
:209A8000203C0221A6790E8002790D101732781EE9F208E4F2781DE2D2E4D25EF20294196C
:209AA000753C01753D00D215129BB4603120E00B30E423EB540F6026B4021B10170201C197
:209AC00085418375822DE52BF07A04758230784212E1AF0289961017E7791102941279132B
:209AE0007824C37A03E29401F250A008DAF7809B20171B30131B7820E2253CF208E2353D64
:209B0000F2500B7B0208E23400F25002DBF7201301227B03785CE6C3953CF6F57B08E6953C
:209B20003DF6427B5007753D00DBF2800608E6427BDBFAE57B7002D21422301310201030CC
:209B4000D23C781DE2D2E4F2D25E029B707B03786016E6F57BB4FF0C0816E6427BB4FF04A2
:209B6000DBF6800608E6427BDBFAE57B7002D2132017137824E22401F2500B7B0308E23481
:209B800000F25002DBF730110E305D0B781DE2D2E4F2D25E740122201502D25DE42212C59F
:209BA000D27582447401F012A7B9D2161292EDC25D0295C712C5D27582447411F030350607
:209BC0000582E0D2E0F0758248301515E53CF42401F0E53DF434001582F0158274FFF0806E
:209BE00008E53CF01582E53DF0E4F52512A7C4D2161292ED1295C77006C25BC25A803320BF
:209C0000E3E720E03230E42FEB30E704D259C25A30E612201504D25B800B205A08205B059D
:209C2000D25A129CE085418375824BE030E706129C3C129C7DEA22C25BC25A223015187594
:209C4000824EE030E711758251E0F42401FC1582E0F43400FD8009758250E0FD0582E0FC43
:209C6000C3E53C9CF53CE53D9DF53D453C6002C25D305908053CE53C7002053D227842209D
:209C80001511E53C26F608E53D36F650050806E6080622E6C3953CF608E6953DF6500F0805
:209CA00016E6B4FF090816E6B4FF03029CE022E5424543454445456003C25A22C25B227878
:209CC0004206E670097E030806E67002DEF922784216E6B4FF137E030816E6B4FF0BDEF868
:209CE000E4F542F543F544F54522128F34D205129D3A305D0F781DE2D2E4F2D25E790E91E4
:209D0000BF0293B7EA601030E427EB540F6008B4081A79080293B790BF3BE030E5085487E8
:209D2000F079070294125487F00293E5D539BB053990BF3BE05487F001A9C2588541837508
:209D4000822E7480F0758206E0602778347A0412E19478207A0412E1947923E9F00582E4DD
:209D6000F030050BD0E0D0E090BF3BE05487F0029412781EE230E33A753C01753D00D21566
:209D800071B4C215602A20E40730E00201C101A9EB30E613205B10D25A91E0790D781EE973
:209DA000F208E4F2029419540F6005B402E001C1D25FE4F527F521532BFC90BF10F005826D
:209DC000F090BF20F00582F090BF247405F08541837582487820E2F53EFCF0158208E2F54A
:209DE0003FF04204081582E2F540F06003B401034C7005790C02943E7582447408F00582E5
:209E0000E054E0F090BF3BE0303D02D2E4300502D2E5F07824E230E002D23B90BF3CF008B1
:209E20000582E2F008E2F57FF59054C020B50254FC6020305F0A753C01753D0071B4C25FE8
:209E4000791030050BD0E0D0E090BF3BE05487F002943E12A7B9E53B702AE53AB420005061
:209E600023302E09753C00753D0412A5143027E6E53A7007E53B7003029F27853A36853B43
:209E800037029EA5C2AF853A36853B37D2AFE536303B0DC23B20E00D153670091537800536
:209EA00030E002153630050B753209201F0E753201800975320B201F0375320312A86F20F0
:209EC00000FD30083B302E08E4F53CF53D12A5143027F2305F0ED215753C01753D0071B444
:209EE000C215C25F30050BD0E0D0E090BF3BE05487F0796975390112A69C12A65C029412F4
:209F0000C3C2AFE53A9536F53AE53B9537F53BD2AF12A5306002C156753B00302E06753D31
:209F2000FF12A5143027F11295C7600530E305C153029FC220E03820E40830050122C25FF0
:209F400001A991BFC25AEB30E602D25B30E502D23F30E712D25D2005E4781DE2D2E4F2D241
:209F60005E790E0293B7540F605AB4021291CF30050BD0E0D0E090BF3BE05487F001C120B4
:209F800005BBB405057911029412B4080791CF79080293B7B40314305F0E753C01753D0055
:209FA000D21571B4C215C25F02A0FCB40190305F0E753C01753D00D21571B4C215C25F02B3
:209FC000A0ED91BFC25AC25D30050122203F0302A0647834792085418375824EE030E74699
:209FE000758251E0F42401F53E1582E0F43400F53F1582E0F43400E3253EF20809E3353FDB
:20A00000F20809E33540F2781DE2D2E4F2305F0F753C01753D00D215129BB4C215C25FD2C0
:20A020005E79100294120582E0F5400582E0F53F0582E0F53EC3E3953EF2F30908E3953F9A
:20A04000F2F315820908E39540F2F3305F12753C01753D00D215129BB4C215C25F0293E517
:20A0600030050A22782079347A0412E19A75390285418375820AE020E009781FE220E603CA
:20A080000293E5128F34D205753C01753D00D215129BB4C215602920E41730E00A90BF3BCF
:20A0A000E05487F00298C190BF3BE05487F00298A9EB30E602D25B540F6005B402E980DD2E
:20A0C000129DB2EA6003303F1590BF3BE030E50879075487F00294125487F00293E5D53981
:20A0E000A2053990BF3BE05487F00298A9796812A6A3D53947AF01D21002A10479E812A625
:20A10000A3D53938303F19783490BF10E0F2080582E0F2A90710100579E8029412029448D4
:20A12000103A0B782079347A0412E19A80E512A65C782079347A0412E19A80D7753C017533
:20A140003D00D215129BB4602220E01520E4030298A9EB540F6014B402F5300504D0E0D073
:20A16000E090BF3BE05487F00298C1128F34029DB2854183758206E0601978347A0412E18D
:20A180009478207A0412E1947923E9F00582E4F002941285418375822EF075820BE030E4C2
:20A1A000057A100295AE30E5057A200295AEE4F527F521532BDC90BF20F00582F090BF102D
:20A1C000F00582F0F560F561303D0790BF3BE0D2E4F0753209201F0375320190BF3C782428
:20A1E000E2F0080582E2F008E2F57FF59054C020B50254FC6005791002943E12C5D2C25D84
:20A2000085418375824879347820E2F3F01582F53EFC0809E2F3F01582F53F42040809E20C
:20A22000F3F540F070084C700D790C02943EB401F8EC70F5D21090BF247407F0853E367540
:20A24000370410100AE53FB404005003853F3712A86F854183758244740AF0D25885363A35
:20A2600085373B2000FD20081EE412A7BE02A2B82000FD300826D224302E09853A3C853B3A
:20A280003D12A5143027F17969300902798912A69C12A65C129CBF029412217AC2AFE536AB
:20A2A000253AF53AE537353BF53BD2AF302E09853A3C853B3D12A51412A530601F853E364A
:20A2C000753704E53FB404005003853F37E53BB4DF0020271650F612A86F8094302E098525
:20A2E0003A3C853B3D12A5143027F11295C7603920E42720E03130E316E4F536F537416967
:20A30000B4050302A405B40306129CBF02A3C702A3D2B407EB7A200295AEEB30E602D25B14
:20A32000540F6005B402EB2188129CBFC25A85418375820AE020E109781FE220E603029337
:20A34000E512A644128F34200505753902D205753C01753D00D215129BB4C215601320E49C
:20A360000620E00B02A3D2EB540F6005B402F52188129DB2EA601130E4EAEB54036009B435
:20A380000333129CBF02A3C790BF3BE020E5065487F00293E5D539085487F07907029412EB
:20A3A000753C01753D00D215129BB4C215601320E40620E00B02A3D2EB540F6005B402F5BD
:20A3C0002188128F3421AE79E812A6A3D5390D029412798B7C0012A6A502944A75210075E9
:20A3E0003C01753D00D215129BB4C215601220E40520E00A80DCEB540F6005B402F6218866
:20A40000128F3421AE75822EE030E006C2E0F002A50FD2E0F07582447411F005827401F0F7
:20A42000058274FFF00582F00582F012A7B9D2161292ED1295C7601720E3F020E40730E066
:20A44000022188808DEB20E70620E63902A50F7582447411F005827401F00582E4F00582D9
:20A46000F0058204F012A7B9D2161292ED1295C7600E20E3F020E40530E002218802A50F3D
:20A48000128F3421AEE4F527F53DF521532BDC90BF10F00582F012C5D27582447408F075EB
:20A4A00082487450F0F53C12A7B9D2161292ED1295C7600B20E3F020E4C330E0C0218812E4
:20A4C0009B9E600B20E3F820E4B330E0B02188E4F527F521532BDC90BF10F00582F012C5B0
:20A4E000D2758244740AF07582487450F53AF0E4F53B12A7BED2161292ED1295C7600B20C2
:20A50000E3F020E40A30E0072188128F3421AE791102941290BF60E53CF0E53D0582F090DB
:20A52000BF637400F074903024027498F0C22E22C3E53E9536F53EE53F9537F53F500215BE
:20A5400040E53E453F454022854183758206E0601278207A0412E1947923E9F00582E4F068
:20A5600002941275820BE030E4057A100295AE30E5057A200295AE12C5D2F5217582447402
:20A5800010F07582487401F0205D08203C0505827480F0D25812A7B9D2161292ED1295C743
:20A5A000605620E0AC20E3EB30E460EB30E602D25B540F603DB4010302A5F2B4020280918D
:20A5C000B407057A200295AEB406057911029412B4050C103C04D23C809D7911029412B4C5
:20A5E000032979E812A6A3D5392E12A63B79E802944AEB30E602D25BC25A129CBF12A63B57
:20A60000305D0312A644D25D0293E5798B12A6A312A63B798B02944A753C01753D00D21584
:20A62000129BB4C215601220E40520E00A80A1EB540F6005B402022188A177793078427A33
:20A640000402E1A812C5D2F5217582447410F012A7B93027FD1295C720E3E922793E7A0387
:20A660008004793C7A02AF017820758220855B83C3E297F009058208DAF7A90722E4F5A083
:20A68000F8FC7A08E2C3CC33CC30E701B3500363049D23DAF008B814E9ECF4227B017C000E
:20A6A00002A6A77C007B05201E0790E410E020E40122781DE24420F290E40EE0FD2401F03E
:20A6C0000582E0FE3400F0E55160E6C0018551A07A50781012E1947810BB0104741C80020B
:20A6E000743CF278127410F2087401F2855B83781488827A0612E184EDF208EEF208EBF2AD
:20A7000008ED4E70047A01800BE9B468057A8002A7147A00E539146003430240EAF2781EB5
:20A72000E9F208ECF2081285A47407F2087407F2BB013378187A0212E194C3855B83758294
:20A74000207936783E7A03E096F7058208DAF8C37582247B03792C7836E6FAE03AF3058206
:20A760000809DBF58046782A8541837582087A0212E184782C7582107A0812E18478347491
:20A780000AF2087404F2E408F2E565C395397837F279387A04784212E1A8793C7403F30945
:20A7A000E4F3784075824B7A1012E18478517958128F0A855BA0D00122E4F53AF53BF53C9B
:20A7C000F53DF525F566305A0E30580B85418375821CE0758226F075240153210390BF649A
:20A7E000E546F090BF65749DF090BF637401F0E54744C0303102C2E690BF62F08541A078B8
:20A8000038E2701D305C277566017405F28541A0783F90A8417A0512E1BF90BF63744380E7
:20A820001B90BF66F07836E20582F090BF6278437A0608E2F0DAFB90BF637442F0855BA0DE
:20A8400022010301340F90BF637402F07400F07403D236F02036FD2290BF68E548303202E6
:20A86000D2E4303002D2E7F090BF697405F02290BF3EE536F42401F0080582E537F4340050
:20A88000F090BF30E532D200F022E4F58CF58A75168075301A90E4027484F075170D90BF5A
:20A8A00080E0F4FF7541E47C0705418541A078101285A490A90512E1E17810E9F2782F7429
:20A8C00001F2781C7404F27826F2782074FFF208F2DCD67551FD7550EC8550A015A0780038
:20A8E0007901E4AC500C05A0F2ECF3140CBCFFF6E4F390BF12F090BF22F074E390BF13F079
:20A9000090BF23F022060416021703185119501A691B6D0012A994E4F5A0F8E230E002D214
:20A920003730E702D25C30E102D23130E502D23020E402D21F20E602D23230E2047410804D
:20A94000027400F57B08E2F404540790BF3BF008E2F54808E2F56508E2F549FC7D00754198
:20A96000E4054185418375822DE52BF0758208E4F00582EDF00D740775822AF008E275828F
:20A9800034F008E2758235F0758245C423F0DCD17524802212E1E712A67DF9E2B5010122CF
:20A9A0007441028D7B90BF357404F090BF007401F0E4F07404F090BF0474A7F0755BE57574
:20A9C000A0E4118A90E402E4F043A80512897890BF35E030E2F675A0E5748179B4F374B468
:20A9E00079DBF3E4F52C12E1E712A67DF9E26975A0E56007D27975490180023114115875A8
:20AA0000A0E5E549700675490102AA1054F870F690D1F612CC8B90D37120B50390D35112AE
:20AA2000CC8B745212CC2490EC7D12CC8B90CF7A12CC8B90D39012CC8B757B017541E590DB
:20AA4000D3FF12CC8BE57B12CE6190D40D12CC8B753903128A9E601730E3041146800630BA
:20AA6000E408D539EE90D419807790D42E807290D41212CC8B12975660028068900000E05E
:20AA80007002806075280112C54690AB6612CC8B75280112C5887583007582087A0812AB6C
:20AAA0005E75280112C54690AB6612CC8B75280112C5887583007582107A1012AB5E752835
:20AAC0000112C54690AB6D12CC8B75280112C5887583007582207A0412AB5EE41242B68034
:20AAE0000312CC8B0541E57BB549005004057B413F90CF7D12CC8B90D3E012CC8B75390251
:20AB0000E4FE90BF80E0F4540F23F890E164E893FDE80493FC74087981F312CE2090D43865
:20AB200012CC8B740A7981F390D39012CC8B90CF7A12CC8B30790C90D4E212CC8B90CF7A66
:20AB400012CC8B90D19112C863787EE26005C26302AB7CD26390CFDD12CC8B02AB7CE012DD
:20AB600042B6A3DAF922202020202C20002C20524556204C4556454C203D200090D5C012F4
:20AB8000C6694110D239753902129583600F20E3F820E05FD539F21039ECD27A2230393942
:20ABA000900000E004FDB40E00500302ABD990000CE0543FF0B410140582E0B40E1BE58207
:20ABC000240DF58274010582058280080582E0042582F582E582B505D875390275640012A5
:20ABE0009523600F20E3F820E007D539F21039E922D27AC2392290CF7A30630390CF9E12F1
:20AC0000CC8B90CF7A30630390D00A12CC8B90D44212CC8B12CCB630730302ACD290CF7AF9
:20AC200030630390CF9E12CC8B90D46012CC8B90D1C812C863787EE2700990CF7A12CC8BF2
:20AC400002ACC079E3E4D2E0D2E1D2E4D2E2D2E3D2E5F390CF7A12CC8B7401B549028009D8
:20AC600090E0B412C863787EE224E4F541F583758234E0F5460582E0F54790CF7A12CC8BBA
:20AC800090E08412C86379E4787EE2F312B78612B91378E779E8E4F2F379E9F379E3E4F31D
:20ACA000C27E207A1B20731875390312ACDA601020E3F830E40AEB20E606D539EE12B9C4A0
:20ACC00030630F90CF7A12CC8B90D44212CC8B12CCB675280112C588E47375390312AD1811
:20ACE000207330207A2D7401127FD512C5D27582447401F012A7B912CEFE2073163027F75F
:20AD00007401127FDAE4F542F543F544F545C25B0295C77401027FDA753910128A9E602AC0
:20AD200020E3F830E41BEB540FB402127AF079FF78FFD8FE12CEFE207315D9F4DAF0D53979
:20AD4000DAD27A75280312C1B4227184207AF222D26730630590CF9E800390CF7A12CC8B4E
:20AD6000D265D26612E1E712A67DF9E26975A0E5607BC265C26690AE017A1475A000780093
:20AD8000E493F2058208DAF875A0E590D4E230633575280112C54690CF7A12CC8B75280146
:20ADA00012C58812CC8B90D44212CC8B12CCB620740330730302B13C90CFBA12CC8B90CF1B
:20ADC000BF12CC8B802775280112C54690CF7D12CC8B75280112C58812CC8B75280112C5C9
:20ADE0004690CF7A12CC8B75280112C58890000075A0E579DC7A14E0F3A309DAFAD2648058
:20AE0000210401070101000001000200030004000500060030630590CFA9800390CF7A12E0
:20AE2000CC8B78DCE2FA30670302AFC5797EEA30E104740080027401F390D85112C8632011
:20AE4000641720740330730302B13C787EE26005EAC2E18003EAD2E1FA797EEA20E004740E
:20AE60000080027401F390D8B112C86320641720740330730302B13C787EE26005EAD2E0F2
:20AE80008003EAC2E0FA797EEA03035401F390D86112C86320641720740330730302B13CAD
:20AEA000787EE27005EAC2E28003EAD2E2FA797EEA30E404740080027401F390D85912C8AA
:20AEC0006320641820740330730302B13C787EE26005EAC2E48003EAD2E4FAEA797EEA2072
:20AEE000E504740080027401F390D88912C86320641720740330730302B13C787EE26005D9
:20AF0000EAD2E58003EAC2E5FA797EEA30E604740080027401F390D87112C8632064172058
:20AF2000740330730302B13C787EE26005EAC2E68003EAD2E6FA797EEA20E7047400800235
:20AF40007401F390D87912C86320641920740330730302B13C787EE26005EAD2E78003EA55
:20AF6000C2E779DCF378DD797EE2F390D86912C86320640F20740330730302B13C787E7983
:20AF8000DDE2F378DF797EE214F30490D88112C86320641020740330730302B13C787E796F
:20AFA000DFE204F378DE797EE2F390D8A112C86320640F20740330730302B13C787E79DE65
:20AFC000E2F302B05478E0797EE2F3F540700675400102AFD954F870F690D89912C8632077
:20AFE000641120740330730302B13C787E79E0E2F3F540756001757BE0057BA87B797EE235
:20B00000F390D96112CC8BE56012CE6190D89112C86320640F20740330730302B13C787E99
:20B02000A97BE2F3057BA87B797EE2F390D96112CC8BE56012CE6190D8A912C86320640F0E
:20B0400020740330730302B13C787EA97BE2F30560D540A520645690000078DC7A14E2F098
:20B06000A308DAFA12A67DF212E24612E1E712A67DF9E26975A0E5601590D52812CC8B3008
:20B08000630990D44212CC8B12CCB602B13CC27930630590CF9E800390CF7A12CC8B30638A
:20B0A0000990D44212CC8B12CCB602AD52C264C26590CF7A12CC8B30630690D00A12CC8BE8
:20B0C00090D1E212C863787EE2607130633390CFF212CC8B90D03812CC8B90CFFA12CC8B04
:20B0E00090D05612CC8B90D00212CC8B90D08112CC8B90D00A12CC8B90D01212CC8B02B1BB
:20B100003420713090CF7D12CC8B90D03812CC8B90CF7A12CC8B90D05612CC8B90CF7A12A8
:20B12000CC8B90D08112CC8B90CF7A12CC8B90D01212CC8B306602D26502AE14C265C2666F
:20B14000C26775280112C588E4737541E579E47401F390D6A212C66975280112C588E47375
:20B1600090CF7D12CC8B30630690CF9E12CC8B90DB4F12CC8B90DBD212CC8B90DBED12CC8C
:20B180008B90DAF512CC8B90DB0C12CC8B90DBF712CC8B90DB4712CC8B90DA9920B503902B
:20B1A000DAA012CC8B90DAA712CC8B90BF80E0F490DB0C30E50390DB1812CC8B90DBFE1299
:20B1C000CC8B90DB4712CC8B90BF80E090DA4620E50390DA4D12CC8B90DA5512CC8B90BFFF
:20B1E00080E0F490DB0C30E60390DB1812CC8B90DC0512CC8B90DB4712CC8B90BF80E0904B
:20B20000DAC520E60390DAD812CC8B90BF80E0F430E70690DB1802B21C90DB0C12CC8B9058
:20B22000DC0C12CC8B90DB4712CC8B90BF80E020E70690DA2402B23B90DA2912CC8B90DA03
:20B240003212CC8B90DB3012CC8B90CF7D12CC8B30631A90D00A12CC8B90D44212CC8B1269
:20B26000CCB630730302B434307202216090CF7D12CC8B30630690CF9E12CC8B90DB4F1287
:20B28000CC8B90DBE012CC8B90DAF512CC8B90BF80E0F430E00690DB1802B29F90DB0C12C3
:20B2A000CC8B90DBF712CC8B747C12CC2490BF80E0F430E10690DB1802B2BE90DB0C12CC76
:20B2C0008B90DBFE12CC8B90DB4B12CC8B90DA6712CC8B90BF80E0F4540F23F890E164E8DA
:20B2E000937E00FDE80493FC74087981F312CE2090D43812CC8B740A7981F390BF80E0F449
:20B3000030E20690DB1802B30C90DB0C12CC8B90DC0512CC8B747C12CC2490BF80E0F490F2
:20B32000DB1820E30390DB0C12CC8B90DC0C12CC8B747C12CC2490BF80E020E41890DB1813
:20B3400012CC8B90DC1312CC8B90DB4712CC8B90DA7202B36A90DB0C12CC8B90DC1312CC49
:20B360008B90DB4712CC8B90DA7712CC8B90DB2412CC8B90DC1A12CC8B90DB4712CC8B904B
:20B38000DA7D12CC8B90BF81E0F490DB1820E10390DB0C12CC8B90DC2112CC8B90DB471228
:20B3A000CC8B90DAEC12CC8B90BF81E0F490DB1820E20390DB0C12CC8B90DC2812CC8B90DE
:20B3C000DB4712CC8B90DAEC12CC8B90BF81E0F490DB1820E30390DB0C12CC8B90DC2F1269
:20B3E000CC8B90DB4712CC8B90DAEC12CC8B90BF81E0F490DB1820E40390DB0C12CC8B907E
:20B40000DC3612CC8B90DB4712CC8B90DAEC12CC8B90DB3012CC8B90CF7D12CC8B306314E7
:20B4200090D00A12CC8B90D44212CC8B12CCB6307202416D75280112C588E47390CF7D30E4
:20B44000630390CF9E12CC8B79E3E3B2E1F390DF7620E10390DF8212CC8B90DF8F12CC8BB1
:20B4600090CF7D12CC8B30630F90D00A12CC8B90D44212CC8B12CCB675280112C588E4731B
:20B4800090CF7D30630390CF9E12CC8B79E3E3B2E4F390DF7620E40390DF8212CC8B90DF57
:20B4A0009C12CC8B90CF7D12CC8B30630F90D00A12CC8B90D44212CC8B12CCB6752801127A
:20B4C000C588E47390CF7D30630390CF9E12CC8B79E3E3B2E2F390DF7620E20390DF82123D
:20B4E000CC8B90DFA812CC8B90CF7D12CC8B30630F90D00A12CC8B90D44212CC8B12CCB618
:20B5000075280112C588E47390CF7D30630390CF9E12CC8B79E3E3B2E3F390DF7620E3034D
:20B5200090DF8212CC8B90DFB512CC8B90CF7D12CC8B30630F90D00A12CC8B90D44212CCE6
:20B540008B12CCB675280112C588E47390CF7D30630390CF9E12CC8B79E3E3B2E7F390DF66
:20B5600076D27E20E705C27E90DF8212CC8B90DFC112CC8B90CF7D12CC8B30630F90D00A75
:20B5800012CC8B90D44212CC8B12CCB675280112C588E47390CF7D30630390CF9E12CC8B73
:20B5A00079E3E3B2E6F390DF7620E60390DF8212CC8B90DFD312CC8B90CF7D12CC8B3063F6
:20B5C0001290D00A12CC8B90D44212CC8B12CCB630720075280112C588E47390CF7D30637E
:20B5E0000390CF9E12CC8B79E3E3B2E079E3F390DF7620E00390DF8212CC8B90DFE312CC50
:20B600008B90CF7D12CC8B30631290D00A12CC8B90D44212CC8B12CCB630720075280112ED
:20B62000C588E47390CF7D30630390CF9E12CC8B79E3E3B2E5F390DF7620E50390DF8212D5
:20B64000CC8B90DFEE12CC8B90CF7D12CC8B30631290D00A12CC8B90D44212CC8B12CCB66D
:20B6600030720075280112C588E47390CF7D30630390CF9E12CC8B90E08412C86379E478F6
:20B680007EE2F375280112C588E47390CF7D30630390CF9E12CC8B79E3E4F375280112C583
:20B6A00088E47390CF7D30630390CF9E12CC8B12B88330630F90CF7D12CC8B90D44212CC1B
:20B6C0008B12CCB675280112C588E47390CF7D30630390CF9E12CC8B78E779E8E4F2F3791D
:20B6E000E9F390CF7A12CC8B7401B54902800990E0B412C863787EE224E4F541F583758248
:20B7000034E0F5460582E0F54712B88378E3E230E6057440F2801454BE7004E220E006905A
:20B72000D46012CC8B90D1C812C863787EE2604E78E3E2603112B78678E3E220E62812B92D
:20B740001378E3E230E007C2E0601B207A1875390312ACE6601020730D20E3F530E407EB50
:20B7600020E603D539EB78E3E4F2C27E30630F90CF7A12CC8B90D44212CC8B12CCB6752832
:20B780000112C588E47378E779E8E4F2F378EA79E9F2F3C27A79E5E4F309F390E13B12CCC9
:20B7A0008B78E5E204F2700608E204F218E2FC08E2FDE4FE740A7981F312CE2078E3E230DC
:20B7C000E10C12B9FF207A2A20732778E3E230E20C12BA61207A1B20731878E3E230E30CF0
:20B7E00012BB31207A0C20730978E3E230E40C12BBCA207A3120732E78E3E230E50C12C059
:20B8000000207A7820737578E3E230E70C12C000207A6920736678E3E230E61312CE87789B
:20B82000E47401F208F2207A5320735078E3E230E00912BCAE207A4420734112CEFE207AF7
:20B840003B20733878E3E230E60690CFF212CC8B90E15112CC8B78E5E2FC08E2FDE4FE742C
:20B860000A7981F312CE2078E5E2F52878E4E2700302B79BC39528600302B79B3073031281
:20B88000A8462278E3E2700790DFFC12CC8B2290E00E12CC8B78E4E2FCE4FDFE740A798176
:20B8A000F312CE2090CF9312CC8B90E03212CC8B78E3E230E10990DF8F12CC8B78E3E23004
:20B8C000E20990DFA812CC8B78E3E230E30990DFB512CC8B78E3E230E40990DF9C12CC8B49
:20B8E00078E3E230E70B90DFC112CC8B78E3E2800C30E50990DFEE12CC8B78E3E230E60947
:20B9000090DFD312CC8B78E3E230E00690DFE302CC8B22C27690E0D912CC8B78E5E2FC082F
:20B92000E2FDE4FE740A7981F312CE2090E0EC12CC8B90E0FC12CC8B78E8E2F52878E7E2A1
:20B940002528F52878EAE22528F52878E9E22528FCE4FDFE7981740AF312CE2090E1151261
:20B96000CC8BE4FEFD78E7E2FC12CE2090E11812CC8BE4FEFD78E8E2FC12CE2090E12012A2
:20B98000CC8BE4FEFD78E9E2FC12CE2090E12812CC8BE4FEFD78EAE2FC12CE2090E132026C
:20B9A000CC8BEB30E702D25930E609301504D25A8002D25B30E502D23F540F603FB4030FCE
:20B9C000305A0122D20FD27A75280712C1B422B4010775280812C1BE22B4020775280312BD
:20B9E000C1B422B4080AD22CD27A75280F12C1B4B407D1D27A75280C12C1BA2202CEFE125D
:20BA0000CEFE20735B90DEBF12CC8B12AD1820734F207A4C75390312ACE6207343207A4032
:20BA2000601020E3F230E438EB20E606D539E831C42279EDE4F3097401F312C2F720732025
:20BA4000207A1D75390312ACE6207314207A11600F20E3F230E409EB20E605D539E831C426
:20BA60002212CEFE20732C90DEEE12CC8B12AD18207320207A1D75390312ACE620731420E5
:20BA80007A11601020E3F230E409EB20E606D539E831C42212C26D79ED740EF3E409F30990
:20BAA000F309F312C2F7207340207A3D12C26D757B3279ED7400F3097420F3E409F309F386
:20BAC00012C2F7207323207A20D57BE675390312ACE6207314207A11601020E3F230E45085
:20BAE000EB20E606D539E831C42212C28279ED740EF3E409F309F309F312C3B120733120CF
:20BB00007A2E780E790012C1F5757B3212C28279ED7400F3097420F3E409F309F312C3B17F
:20BB200020730D207A0A7800792012C1F5D57BDC2212CEFE20732C90DF0012CC8B12AD184E
:20BB4000207320207A1D75390312ACE6207314207A11601020E3F230E409EB20E606D5394D
:20BB6000E831C42279ED7400F3097420F3E409F309F312C2F7207351207A4E12C2A12073EE
:20BB800048207A4575390312ACE620733C207A39601020E3F230E431EB20E606D539E831BF
:20BBA000C422753C01753D0012C48820731B207A18753C01753D0012C48820730C207A0979
:20BBC00020590675281412C1B42212CEFE20735890DED112CC8B12AD18207A4C207349750D
:20BBE000390312ACE620731B207A18601720E3F230E410EB20E60DD539E831C422207303D4
:20BC0000307A012279ED740EF3E409F309F309F312C2F72073ED207AEA79ED740EF3E4090D
:20BC2000F309F309F312C2F7207329207A2612C2A1207320207A1D75390312ACE6207314F7
:20BC4000207A11601020E3F230E409EB20E606D539E831C422753C02753D0012C48820735D
:20BC600042207A3F30590775281012C1B422753C01753D0012C488207329207A2620590705
:20BC800075281412C1B422D215753CFF753DFF12C488C21520730C207A092059067528145B
:20BCA00012C1B42212CEFE207303207A002212CEFE207341207A3E90DF2812CC8B12C26DE0
:20BCC00090BF20E4F005827400F090BF247401F0753300753404753500793375370275365A
:20BCE00000753203D2AA128E5E2000FD30080775281D12C1B02212C28290BF20E4F0058245
:20BD00007400F090BF247403F07532017933128E5E2000FD30080775281E12C1B02278005F
:20BD2000790212C1F512C28290BF20E4F005827400F090BF247401F0753300753404753565
:20BD4000007933753702753600753203D2AA128E5E2000FD30080675281D12C1B022FFFF02
:20BD6000FFFFFFFFFFFFFFFFFFFFFFFFFFFFFFFFFFFFFFFFFFFFFFFFFFFFFFFFFFFFFFFFE3
:20BD8000FFFFFFFFFFFFFFFFFFFFFFFFFFFFFFFFFFFFFFFFFFFFFFFFFFFFFFFFFFFFFFFFC3
:20BDA000FFFFFFFFFFFFFFFFFFFFFFFFFFFFFFFFFFFFFFFFFFFFFFFFFFFFFFFFFFFFFFFFA3
:20BDC000FFFFFFFFFFFFFFFFFFFFFFFFFFFFFFFFFFFFFFFFFFFFFFFFFFFFFFFFFFFFFFFF83
:20BDE000FFFFFFFFFFFFFFFFFFFFFFFFFFFFFFFFFFFFFFFFFFFFFFFFFFFFFFFFFFFFFFFF63
:20BE0000FFFFFFFFFFFFFFFFFFFFFFFFFFFFFFFFFFFFFFFFFFFFFFFFFFFFFFFFFFFFFFFF42
:20BE2000FFFFFFFFFFFFFFFFFFFFFFFFFFFFFFFFFFFFFFFFFFFFFFFFFFFFFFFFFFFFFFFF22
:20BE4000FFFFFFFFFFFFFFFFFFFFFFFFFFFFFFFFFFFFFFFFFFFFFFFFFFFFFFFFFFFFFFFF02
:20BE6000FFFFFFFFFFFFFFFFFFFFFFFFFFFFFFFFFFFFFFFFFFFFFFFFFFFFFFFFFFFFFFFFE2
:20BE8000FFFFFFFFFFFFFFFFFFFFFFFFFFFFFFFFFFFFFFFFFFFFFFFFFFFFFFFFFFFFFFFFC2
:20BEA000FFFFFFFFFFFFFFFFFFFFFFFFFFFFFFFFFFFFFFFFFFFFFFFFFFFFFFFFFFFFFFFFA2
:20BEC000FFFFFFFFFFFFFFFFFFFFFFFFFFFFFFFFFFFFFFFFFFFFFFFFFFFFFFFFFFFFFFFF82
:20BEE000FFFFFFFFFFFFFFFFFFFFFFFFFFFFFFFFFFFFFFFFFFFFFFFFFFFFFFFFFFFFFFFF62
:20BF0000FFFFFFFFFFFFFFFFFFFFFFFFFFFFFFFFFFFFFFFFFFFFFFFFFFFFFFFFFFFFFFFF41
:20BF2000FFFFFFFFFFFFFFFFFFFFFFFFFFFFFFFFFFFFFFFFFFFFFFFFFFFFFFFFFFFFFFFF21
:20BF4000FFFFFFFFFFFFFFFFFFFFFFFFFFFFFFFFFFFFFFFFFFFFFFFFFFFFFFFFFFFFFFFF01
:20BF6000FFFFFFFFFFFFFFFFFFFFFFFFFFFFFFFFFFFFFFFFFFFFFFFFFFFFFFFFFFFFFFFFE1
:20BF8000FFFFFFFFFFFFFFFFFFFFFFFFFFFFFFFFFFFFFFFFFFFFFFFFFFFFFFFFFFFFFFFFC1
:20BFA000FFFFFFFFFFFFFFFFFFFFFFFFFFFFFFFFFFFFFFFFFFFFFFFFFFFFFFFFFFFFFFFFA1
:20BFC000FFFFFFFFFFFFFFFFFFFFFFFFFFFFFFFFFFFFFFFFFFFFFFFFFFFFFFFFFFFFFFFF81
:20BFE000FFFFFFFFFFFFFFFFFFFFFFFFFFFFFFFFFFFFFFFFFFFFFFFFFFFFFFFFFFFFFFFF61
:20C0000012CEFE20733390DF3F307E0390DF5212CC8B12AD18207321207A1E75390312AC41
:20C02000E6207315207A12601120E3F230E40AEB20E607D539E812B9C422E4F55CF55DF527
:20C040005EF55F79F9F312C26D79ED7400F3097420F3E409F309F312C2F72073DC207AD9A2
:20C06000785CE62401F650097A0308E63400F6DAF9207E0978F9E204F270CE8003305BC925
:20C08000785F7A04C3E613F618DAFA75390312ACE6207315207A12601120E3F230E40AEB95
:20C0A00020E607D539E812B9C42275210012C5D2758244740CF0758248E55CF01582E55D99
:20C0C000F01582E55EF012A7B912CEFE207A0E20730B3027F41295C7700402C11922785C11
:20C0E000E6F53C08E6F53D453C7006753CFF753DFF12C4882073E6207AE3785CE6C3953C0F
:20C10000F608E6953DF67A0208E69400F6DAF9785C7A04E670C808DAFA75210012C5D275AC
:20C120008244740CF07582487401F012A7B912CEFE207A0E20730B3027F41295C770040260
:20C14000C185227942785CE7F6F53C0809E7F6F53D0809E7F60809E7F6D21512C488C215C2
:20C1600020734C207A49785CE6C3953CF608E6953DF67A0208E69400F6DAF9785C7A04E604
:20C1800070D708DAFA305A0775281512C1B422D215753C01753D0012C488C215207310204D
:20C1A0007A0D205A0775281712C1B4227521002279EA800CD27A79E7800679E9800279E8FC
:20C1C000C0E0E304F3E528142390DC8F2582F58250020583307A02C276D27C75280112C507
:20C1E0004690DC3D12CC8B75280112C58812CC9EC27CD0E022900000752801E0C395287060
:20C200000BA30528D8F5E96002D9F022797EE528F375280112C54675281331BED27C90DC35
:20C220004E12CC8B75280112C588E582FCE583FDE4FE12CE2075280112C54690DC5D12CC3E
:20C240008B75280112C58879817410F3E0FCE4FDFE12CE2090DC6B12CC8B787EE2FCE4FD35
:20C26000FE12CE2090CF7A12CC8BC27C2278007920900000752801E528F0A30528D8F8D969
:20C28000F62278007920900000E4F0A3D8FBD9F92278007920900000E528F0A3D8FAD9F8C3
:20C2A000227401127FD575210012C5D27582447410F07582487401F012A7B912CEFE207A05
:20C2C000282073253027F47401127FDA1295C7600C20E3CD20E00930E40C12B9A2029CBFB6
:20C2E00075280331B42212B9C47401127FDA22752100C25D02A7B97401127FD5856539E40D
:20C30000F527532BFCF52190BF10F00582F0F560F56112C5D275824878EDE2F53AF015821B
:20C3200008E2F0F53B758244740AF0E412A7BE12CEFE207363207A603027F47401127FDAF6
:20C340001295C7605920E3E330E00675280331B42230E44112B9A2205B3E207A3B200A4B4E
:20C36000D5390302C395D215753CFF753DFF12C488C2153027FD1295C7601820E3E830E49C
:20C3800014EB30E61079E8E304F312CEFE207308207A05809612B9C47401127FDA22C25963
:20C3A000C25A753C01753D0002C50A75280C31BA227401127FD5E4F527532BFCF52190BFBC
:20C3C00010F00582F012C5D275824878EDE2F53CF0158208E2F53DF07582447408F012A793
:20C3E000B912CEFE20733D207A3A3027F47401127FDA1295C77010C259C25A753C01753D4E
:20C400000012C50A02C47F20E3D420E00720E40A12B9C42275280331B42212B9A2C259C268
:20C420005A302C067401127FDA22207AF7753C01753D0012C50A12CEFE207A0F20730C3012
:20C44000590AC259D25D75281031B422C25D303F2E854183758247E030E71278F190BF1067
:20C46000E0F2080582E0F275281131B42278F190BF10E0F2080582E0F275281231B42278AB
:20C48000ED79F17A0402E19A7401127FD512C5D27582447411F0758248301517E53CF42442
:20C4A00001F01582E53DF43400F0158274FF3400F08008E53CF01582E53DF0E4F52512A793
:20C4C000C412CEFE20732A207A273027F47401127FDA1295C7602620E3E120E00F30E417FF
:20C4E00012B9A2302C1175280F31B42275280331B47401127FDA2220590B205B0B301508D1
:20C50000C25B02C5232015F8C25A7842E6253CF608E6353DF6500B7B0208E63400F650023C
:20C52000DBF7227842E6C3953CF608E6953DF650147B0208E69400F6500BDBF7E4F542F591
:20C5400043F544F54522A983A88290E5B4E0F582304006A3E8F0A3E9F0304203A3EAF0309E
:20C560004303A3EBF0304403A3ECF0304503A3EDF0304603A3EEF0304703A3EFF0E5827537
:20C5800082B4F08983888222A983A88290E5B4E0F582304704E0FF1582304604E0FE158287
:20C5A000304504E0FD1582304404E0FC1582304304E0FB1582304204E0FA1582304008E07B
:20C5C000F91582E0F81582E5827582B4F08983888222854183758245E054E0F07A04058294
:20C5E000E4F00582DAFB227800752800BB01012274FF8B28C2AF8528F08485F028D2AFC55A
:20C600002804FA6B70030528FAAF28EE8B28C2AF8528F08485F028D2AFF9AE28D2108F285F
:20C62000EEC2AF8528F0A485F028D2AF28F8EE8A28C2AF8528F0A485F028D2AFAE282D5059
:20C64000010E8B28C2AF8528F08485F028D2AF28F8AD28EE70C8101007E9FEECFDE8FC2250
:20C66000AE28ECFDE4C8FC80B57A0C79DBE3F808E581F27472F58108D0E0F2DAFAE8F375DF
:20C680008166752801B146752801B14690CF7A12CC8B752801B188306310752801B14690A8
:20C6A000CF9E12CC8B752801B18812CC9EE582240650020583F582E49370EFE582240650B8
:20C6C000020583F582E493797EF330633990CFF212CC8B90D03812CC8B90CFFA12CC8B901F
:20C6E000D05612CC8B90D00212CC8B90D08112CC8B90D00A12CC8B90D0B312CC8B90D1677F
:20C7000012CC8B02C73920712A90CF7D12CC8B90D03812CC8B90CF7A12CC8B90D05612CCD7
:20C720008B90CF7A12CC8B90D08112CC8B90CF7A12CC8B90D15312CC8B752801B14690D18D
:20C740008012CC8B752801B188752801B14690D18412CC8B752801B188787EE212CC247510
:20C760002801B14690D18912CC8B752801B188752801B14690D18B12CC8B752801B188129C
:20C78000CCB6307102C1CA20720920740330730602C84702C8377875E27006787EE202C716
:20C7A000A7B40120786CE2797EF3B4780302C847752801B188752801B146787EE2F812CEF1
:20C7C000E630696190D4A330632112CC8B90E56C12CC9590D4D012CC8B90D44212CC8B1243
:20C7E000CCB690CFBA12CC8B02C837752801B14690CF7D12CC8B752801B18812CC8B75287D
:20C800000112C54690D4D012CC8B75280112C58875280112C54690CF7A12CC8B75280112B3
:20C82000C58802C837C083C08290C83775280112C546E490C8407375280112C58802C682A5
:20C840007403D082D0837375280112C5887581667A0C78DBE2F9E319C0E0DAFAE319F5815A
:20C86000E9F22275287D12C54612CC9E20650B797E740693F309740593F37402937980F384
:20C88000740793FB740393F8740493F58288837880E2B4020302CA2475280112C54690D161
:20C8A0008012CC8B75280112C5887880E2B4011A740A7981F375280112C54690D43D12CC44
:20C8C0008B75280112C58802CA12B40470E4937981F37400FE740193FD740293FC12CE20EA
:20C8E00075280112C54690D18F12CC8B75280112C5887400FE740393FD740493FC12CE20A7
:20C9000075280112C54690D18312CC8B75280112C5883063007400FE787FE2FD18E2FC122F
:20C92000CE203063007881E2B4080990D43812CC8B02CA1290D43D12CC8B02CA12B40857F8
:20C9400075280112C54612CC9EA3A3E493601475280112C54690CF9112CC8B75280112C5E6
:20C960008880E375280112C54690D18312CC8B75280112C58830630075280112C588787E41
:20C98000E223F528E582252850020583F58212CC9E30630002CA1275280112C54690DA1C42
:20C9A00012CC8B75280112C58875280112C54690CF9112CC8B75280112C58875280112C58B
:20C9C0004690DA1E12CC8B75280112C58875280112C54690D18312CC8B75280112C58830EE
:20C9E0006300787EE2B4011575280112C54690DA1C12CC8B75280112C58802CA0F75280112
:20CA000012C54690DA1E12CC8B75280112C58830630075280112C54690D18912CC8B7528CD
:20CA20000112C58875280112C54690D18B12CC8B75280112C588206436306312752801127A
:20CA4000C54690CFB512CC8B75280112C58812CCB620711B20721820771520731220740F73
:20CA600020720C7875E26007CBC39B5005D26802CB3675287D12C58875287D12C546740300
:20CA800093F8740493F58288837880E2B4010F12CDB430690302CB368D28EC02CB2FB40459
:20CAA0003912CDB4206918EE7013ED740193C39D400F7009740293C39C40066004D26A80AD
:20CAC00075740393C39D40F5700B740493C39C5004D26A80618D28EC8055B40846E4FCC0D4
:20CAE00082C083E4937009D269D083D08202CB36F8740193F58288837875E2FBE4F9E993F9
:20CB00006017FAE9246CF8E2C39A700D09DBEFD083D082752800EC8016D083D082A3A30CE9
:20CB200002CADFB41009786CE212CED6752800797EF309E528F375287D12C5887528011248
:20CB4000C546207113207210206925206822206A1975280112C5882230630690CFBF12CCD5
:20CB60008B75280112C58802C86390D4B702CB7390D4A330632012CC8B90E56C12CC95909E
:20CB8000D4D012CC8B90D44212CC8B12CCB690CFBA12CC8B80C275280112C54690CF7D1278
:20CBA000CC8B75280112C58812CC8B75280112C54690D4D012CC8B75280112C588752801C5
:20CBC00012C54690CF7A12CC8B75280112C58802CB5812897890BF35E030E2F622C082C031
:20CBE000837402127FD512897890BF35E030E1F690BF34E0547FF52805827402F012897805
:20CC000090BF35E020E1F690BF35E4F07402127FDAD083D082E528B441004007B45A005034
:20CC20000224202212CC28E4207C0430760122C083C082C000F5287401127FD5E52890BFA0
:20CC400034F005827401F012897890BF35E020E01F30E1F390BF34E005827402F0128978C7
:20CC600090BF35E020E1F690BF35E4F0E52880CE90BF35E4F012897890BF35E020E0F6746D
:20CC800001127FDAD000D082D08322E4939128E528A370F722E09128E528A370F8227528B8
:20CCA0000112C546E493F8740193F5828883918B75280102C58875280C12C54690E56C7934
:20CCC0006BE4F3752D00752E0071DDB47F22796BE360F630630512CD9B80EE207004745C29
:20CCE00091241582E09124796BE314F3D27080D91070028006FB745C9124EBB40D05E4F0DD
:20CD000002CD89B4031575280112C54690CF85918B75280112C588D2738079B4152220638B
:20CD200015D27175280112C54690CF8B918B75280112C588805E796BE3608E12CD9B80F65A
:20CD4000B41707306302D272804AB41A1575280112C54690CF88918B75280112C588D2747A
:20CD60008032B40A04D277802BF528C39420500302CCC9796BE3C3940850F5796BE304F3A4
:20CD8000E528F0A3912402CCC9740D9124758275796BE3F075280C12C5882275280112C5AF
:20CDA0004690CF96918B75280112C588796BE314F315822275280D12C5467400FEFDFC90D6
:20CDC000E56CE0603BF528C3943040327881E2B40807E528C394378005E528C394394004D2
:20CDE0006002801AE528C39430F52812CE06EC2528FCED3400FDEE3400FE058280C4D26927
:20CE000075280D02C5887881E2FBE4FAF9F8E82CF8E93DF9EA3EFADBF5E8FCE9FDEAFE2283
:20CE20007528FD12C54690E576E47808F0A3D8FC7881E2FB12C5E7E5281582F0EE70F5ED1D
:20CE400070F2EC70EF90E576C26C7808E012CE61A3D8F9206C04743091247528FD12C58815
:20CE600022C082C0837003306C0890CE77939124D26CD083D08222303132333435363738FE
:20CE80003961626364656612CEFE207348207A4590DF11918B90CF7A918B85418375825249
:20CEA000E02408FF757B0885418375824BE0C4540FD161E0540FD161C082D57B0A757B08A2
:20CEC00090CFD3918B800590CF81918BD0828541830582DFD822B4790474018008B46E0335
:20CEE000E48002D269227402936010B5000122E582240650020583F58280EBD2692278E319
:20CF0000E230E002C2E0D27BC273C274C27590BF31E0F030E22590BF35E030E11E90BF34EF
:20CF2000E0F52805827402F012897890BF35E020E1F690BF35E4F0E528800302CF76C27B2D
:20CF4000B40307D27390CF85818BB41A09D274D27390CF88818BB40F14B27630760AC276A2
:20CF600090D13A918BD2762290D147818BB4140620270302B913C27B22320D0A000D0A0A2D
:20CF8000000A0808005E63005E7A005E75005E74002F002C200008200800203D20001B5B9B
:20CFA000324A1B5B303B3048001B5B303B3048001B5B304A001B5B304B001B5B324B001B54
:20CFC0005B3141001B5B3241001B5B3341001B5B3441001B5B37412020202020001B5B3092
:20CFE0006D001B5B31373B3048001B5B31383B3048001B5B32303B3048001B5B32313B30D2
:20D0000048001B5B32323B3048001B5B32333B3048003C63723E2020202D2057696C6C20F9
:20D02000656E746572207468652064656661756C742076616C756500006374726C2F6820C3
:20D040002D204E6F7420696D706C656D656E74656420796574006374726C2F63202D205226
:20D06000657475726E7320796F7520746F207468652070726576696F7573206C6576656C59
:20D08000006374726C2F75202D2044656C657465732063757272656E7420696E7075742071
:20D0A0006966206E6F203C63723E20656E7465726564006374726C2F77202D2052657772C6
:20D0C000697465732073637265656E206F722070726F6D7074006374726C2F74202D204F24
:20D0E00075747075747320746573742070726F677265737320616E642063757272656E7490
:20D100002073756D6D617279006374726C2F6F202D2053746F707320616E642073746172DB
:20D120007473206F757470757420746F20746865207465726D696E616C000D0A4F75747098
:20D140007574206F6666000D0A4F7574707574206F6E000D0A0A53656C6563742066756EFC
:20D160006374696F6E20001B5B31383B31304853656C6563742066756E6374696F6E2000A9
:20D180002028002C6465663D002900203A20002D00D19908D1BF0001010D0A566964656FCD
:20D1A00020646973706C6179206F722068617264636F7079207465726D696E616C2000D171
:20D1C000C4D1C60076006800D1D01000000000010D0A41726520796F752073757265203F7A
:20D1E0002000D1EA1000000000010D0A4D6F64696679203F20000D0A0A0A0A0A0A0A0A0ADE
:20D200000A0A0A0A0A0A0A0A0A0A0A0A0A0A0A0A0A0A20202020202020202020202020209A
:20D22000202020202A2A2A2A2A2020202A2A2A2A2A2020456D756C657820436F72706F7225
:20D240006174696F6E0D0A20202020202020202020202020202020202020202020202A2072
:20D260002A202020202020203335343520486172626F7220426F756C65766172640D0A205A
:20D2800020202020202020202020202020202020202A2A2A2A2A202A202A2A2A2A2A202020
:20D2A000502E4F2E20426F7820363732350D0A2020202020202020202020202020202020FF
:20D2C0002020202020202A202A20202020202020436F737461204D6573612C2043612C205E
:20D2E00039323632360D0A2020202020202020202020202020202020202A2A2A2A2A2020BC
:20D30000202A2A2A2A2A20202837313429203636322D353630300D0A202020202020202021
:20D32000202020202020202020202045204D2055204C204520580D0A0A0A20202020202032
:20D3400020202020202020202020202020202020002020202020554331372F3138204669C6
:20D36000726D77617265207265766973696F6E20002020202020554330372F382046697229
:20D380006D77617265207265766973696F6E20000D0A202D2D2D2D2D2D2D2D2D2D2D2D2D42
:20D3A0002D2D2D2D2D2D2D2D2D2D2D2D2D2D2D2D2D2D2D2D2D2D2D2D2D2D2D2D2D2D2D2DCD
:20D3C0002D2D2D2D2D2D2D2D2D2D2D2D2D2D2D2D2D2D2D2D2D2D2D2D2D2D2D2D2D2D2D00DA
:20D3E0002020202020436F6E74726F6C6C6572204373722061646472657373203D20000D91
:20D400000A20202020447269766520230020697320004F6E6C696E65004F66666C696E6501
:20D42000206F72206E6F74207265616479006E6F7420746865726500206F6374002064656D
:20D4400063005072657373203C63723E20746F20636F6E74696E75652E2E2E1B5B304B00EA
:20D460000D0A0A2A205741524E494E47202A2C207573652073637261746368207461706576
:20D48000206F6E6C792C2064617461206F6E20746170652077696C6C206265206C6F73745C
:20D4A0000D0A0007496E76616C696420726573706F6E73652C2000074F7574206F662072E6
:20D4C000616E676520726573706F6E73652C200020506C656173652072652D656E7465721A
:20D4E000200007556E70726F6772616D6D6564206F7220636F72727570746564206E6F76A8
:20D5000072616D2C2000070D0A0A4572726F72206F6E2072656164206E6F7672616D20635E
:20D520006F6D6D616E642000070D0A0A4572726F72206F6E207772697465206E6F7672618F
:20D540006D20636F6D6D616E6420000D0A0A546573742070726F6D707420312C20656E74D8
:20D5600065722079206F72206E2C206465663D793A20000D0A0A546573742070726F6D7012
:20D580007420322C20656E7465722079206F72206E2C206465663D6E3A20000D0A52657372
:20D5A000706F6E73652077617320796573000D0A526573706F6E736520776173206E6F009C
:20D5C000D5EBFF02D5C3D6276102ABF6D6376402AD50D6516E02AD52D66A7402B14AD684E0
:20D5E0007302B16000000002D5E7610D0A2020202020202020202020202020202020204DE2
:20D6000041494E204D454E550D0A2020202020202020202020202020202020203D3D3D3D92
:20D620003D3D3D3D3D0A000D0A61202D20416C6C207465737473000D0A64202D2044726957
:20D64000766520636F6E66696775726174696F6E000D0A6E202D204E6F7672616D206D6104
:20D66000696E74656E616E6365000D0A74202D20546573742073656C656374696F6E206DEA
:20D68000656E75000D0A73202D20446973706C6179207377697463682073657474696E67A5
:20D6A0007300D6FDFF02D6A5D7436202B43CD7587702B4C4D7696602B508D7797302B480BC
:20D6C000D7957002B624D7A76502B54CD7C07202B594D7D46802B5DBD7EA6C02B66BD7FB91
:20D6E0006402B6A3D8146302B68BD82B6702B6CCD8347802D6F300000002D6F9780D0A201C
:20D70000202020202020202020202020546573742053656C656374696F6E204D656E750D61
:20D720000A202020202020202020202020203D3D3D3D3D3D3D3D3D3D3D3D3D3D3D3D3D3DF5
:20D740003D0A000D0A62202D20426F7420616E6420726577696E64000D0A77202D205772B7
:20D760006974652F72656164000D0A66202D2046696C65206D61726B000D0A73202D20531D
:20D780007061636520666F72776172642F72657665727365000D0A70202D20506F736974AD
:20D7A000696F6E696E67000D0A65202D20506F736974696F6E696E6720746F20456F74001E
:20D7C0000D0A72202D20526571756573742073656E7365000D0A68202D20486F7374206D15
:20D7E000656D6F727920646D61000D0A6C202D204C6F6F7020636F756E74000D0A64202D10
:20D8000020446973706C61792073656C656374696F6E73000D0A63202D20436C65617220CB
:20D8200073656C656374696F6E73000D0A67202D20476F000D0A78202D20457869742074E4
:20D84000686973206D656E7500D8B904DA1700000AD991100000000101D8B9100000000101
:20D8600001D8C808DA12000101D8E804DA17000101D901100000000101D9C81000000000BD
:20D8800001D91F04DA08000002D9AA100000000001D96B04DA0D000001D94104DA170001D3
:20D8A00001D97104DA0D000701D98504DA0D000001D9F01000000000010D0A416461707405
:20D8C00069766520646D61000D0A557365632064656C6179206265747765656E20646D6180
:20D8E00020627572737473000D0A416461707469766520646D61207468726573686F6C64E1
:20D90000000D0A456E61626C6520736373692070617269747920636865636B696E67000DB5
:20D920000A4D617820726574727920636F756E7420666F722074617065206572726F72732A
:20D94000000D0A4E756D626572206F662064726976657320746F20636F6E666967757265C0
:20D96000000D0A447269766520230020692E642E000D0A5363736920616461707465722040
:20D98000692E642E00204C756E206E756D626572000D0A456E61626C6520736373692064B2
:20D9A0006973636F6E6E656374000D0A456E61626C65207363736920736C6F772063616246
:20D9C0006C65206D6F6465000D0A456E61626C652073796E6368726F6E6F757320736373FF
:20D9E00069207472616E73666572206D6F6465000D0A50726576656E74206D656469612039
:20DA000072656D6F76616C000A0000000A0A00000007DA20DA22000A0001000779006E00FC
:20DA2000320034004C6F6F7000436F6E74696E756500206F6E2073656C66207465737420DA
:20DA40006572726F7200456E61626C650044697361626C650020666173742066696C6520F3
:20DA60007365617263680041646472657373203D20004D73637000546D7363700020556E70
:20DA80007265616461626C652068617264776172652073776974636800554330372F3800D0
:20DAA000554331372F3800207363736920636F6E74726F6C6C65722072657365742073777C
:20DAC0006974636800456E61626C652073637369207265736574730044697361626C6520FB
:20DAE0007363736920726573657473004E6F742075736564000D0A205F5F5F5F5F5F5F20CC
:20DB00000D0A7C202020202020207C000D0A7C205B2A20205D207C000D0A7C205B20202A2D
:20DB20005D207C000D0A7C205B2020205D207C000D0A7C202020202020207C0D0A202D2D05
:20DB40002D2D2D2D2D20002D2D20007C2D2000202020202020202020202020202020202061
:20DB600046756E6374696F6E732073656C656374656420627920696E6469636174656420A3
:20DB80005377697463682073657474696E67730D0A2020202020202020202020202020208B
:20DBA00020202D2D2D2D2D2D2D2D2D2D2D2D2D2D2D2D2D2D2D2D2D2D2D2D2D2D2D2D2D2DDF
:20DBC0002D2D2D2D2D2D2D2D2D2D2D2D2D2D2D2D2D000D0A0A53776974636820312F320003
:20DBE0000D0A0A53776974636820332F340D0A206F6666206F6E00202D2031202D00202D35
:20DC00002032202D00202D2033202D00202D2034202D00202D2035202D00202D2036202DAB
:20DC200000202D2037202D00202D2038202D00202D2039202D00202D3130202D00070D0AF5
:20DC40000A2A2A204552524F52202A2A20000D0A202061646472657373203A20002C2041E4
:20DC6000435455414C2020203A20002C204558504543544544203A20002C205245434F5292
:20DC8000442053495A45203A20002048455800DCCBDCCBDCD7DCCBDCCBDCCBDCE7DCFBDDF9
:20DCA00016DCCBDCCBDD2CDD53DD70DD8CDD9CDDB7DDD2DDE9DDF9DE10DE2BDE46DE63DE7F
:20DCC00072DE88DCCBDCCBDE94DEA0626164206D65737361676500556E6974206E6F7420D1
:20DCE0006F6E6C696E650048617264206572726F72207265706F7274656400436F72726556
:20DD0000637461626C65206572726F72207265706F727465640050617269747920657272E7
:20DD20006F72207265706F7274656400546170652077726974652070726F746563746564BE
:20DD40002C206E6F742073637261746368207461706500496E76616C696420627974652099
:20DD6000636F756E7420666F7220777269746500496E76616C6964206279746520636F75C6
:20DD80006E7420666F72207265616400426C616E6B2074617065207265616400556E657870
:20DDA00070656374656420656F6620656E636F756E74657265640052656164207461706592
:20DDC000207265636F7264207472756E636174656400526561642074617065207265636FAB
:20DDE00072642073686F72740044617461206D6973636F6D70617265004578706563746565
:20DE00006420656F66206E6F7420666F756E6400556E657870656374656420626F74206598
:20DE20006E636F756E746572656400556E657870656374656420656F7420656E636F756E86
:20DE4000746572656400457870656374656420626F74206E6F7420656E636F756E746572B3
:20DE600065640054617065206E6F7420626C616E6B0054617065206D61726B206E6F7420D0
:20DE80007772697474656E004472697665206572726F7200446D6120746F20686F7374003E
:20DEA000446D612066726F6D20686F7374000D0A5465737420636F6D706C6574650A000D57
:20DEC0000A426F742F726577696E642074657374000D0A537061636520666F727761726463
:20DEE0002F726576657273652074657374000D0A57726974652F726561642074657374004A
:20DF00000D0A46696C65206D61726B2074657374000D0A526571756573742073656E736581
:20DF200020646174610D0A000D0A486F7374206D656D6F727920646D612074657374000D63
:20DF40000A506F736974696F6E696E672074657374000D0A506F736974696F6E696E67207A
:20DF6000746F20456F7420746573740020636F6D706C657465000D0A456E61626C65642C2F
:20DF800020000D0A44697361626C65642C2000426F742F726577696E640D0A00537061636B
:20DFA0006520662F720D0A0057726974652F726561640D0A0046696C65206D61726B0D0A6F
:20DFC00000506F736974696F6E20746F20456F740D0A00526571756573742073656E736563
:20DFE0000D0A00486F737420646D610D0A00506F736974696F6E696E670D0A004E6F207408
:20E0000065737420656E61626C65640D0A000D0A54657374732073656C6563746564206699
:20E020006F72206C6F6F7020636F756E74206F6620000D0A2D2D2D2D2D2D2D2D2D2D2D2D94
:20E040002D2D2D2D2D2D2D2D2D2D2D2D2D2D2D2D2D2D2D2D2D2D2D2D2D2D2D2D2D2D2D2D20
:20E060002D2D2D2D2D2D2D2D2D2D2D2D2D2D2D2D2D2D2D2D2D0D0A0A00517569636B20743D
:20E0800065737400E08C04E0AF0001030D0A456E746572206E756D626572206F66206C6F83
:20E0A0006F707320746F2065786563757465000A000000FFE0BC04E0D40001010D0A456ECF
:20E0C000746572206472697665202320746F2074657374000A000100070D0A0A45786563DD
:20E0E0007574696E67207061737320000D0A546573742073756D6D6172793A000D0A20208C
:20E10000546F74616C2023206F66206572726F7273203D200020280020486172642C200056
:20E1200020536F66742C2000204465766963652C200020446D61290D0A0A000D0A0A2D2D24
:20E140003E205374617274206F66207061737320000D0A2D2D3E20456E64206F662070619B
:20E1600073732000F940E104E108E10CE124E128E12CE144E148E14CE150E154E158E15C33
:20E18000E160E164E0F2058208DAF922E2F0058208DAF922E4F208DAFC22E2F30809DAFABD
:20E1A00022E2F70809DAFA22E6F30809DAFA22E6F0080582DAF922E0F7058209DAF922E4E3
:20E1C00093F2A308DAF92205A0E4F8F2D8FD22E4A393F9E2F3A3E493F870F422E4A393F224
:20E1E000A3E493F870F622E4F5A0F8F97A15800975A001780079187A80C210C21112E2C68B
:20E2000074A012E27FE912E27F12E2C674A1D21012E27F7B08C3D29712E2D5A29633C297BB
:20E2200012E2D5DBF1F2BA0102800CC296D29712E2D5C297D29608DADAC296D29712E2D57D
:20E24000D29612E2D522E4F5A0F8F97E03800975A001780079187E10C210C21112E2C67477
:20E26000A012E27FE912E27FD2117A08E212E27F7C167B00DBFEDCFCE92408F9DEDC227B52
:20E2800008C3C29733929612E2D5D29712E2D5DBF1C297D29612E2D5D2977D0030960ADD1B
:20E2A000FB744A759000028D7B12E2D5C2971010127D00209604DDFB80E730110808E2DABF
:20E2C000BE4139D29622D296D29712E2D5C29612E2D5C297227C02DCFE22E0F57C12E8E0A1
:20E2E000E57D6003028D7B90BF247401F0E4F535F534E57C700C7533807B007AB490E5F22B
:20E300008029E4F53775360875338090E49475A0007800E493F208A3B808F812E44D75341C
:20E320000275337E7B017A5690E49C8B378A3675A00078000BE493F2A308B8000205A0DAF2
:20E34000F4DBF212E474E57C900008600975823F30B50353051FECF0A3EDF030B502807167
:20E36000E57C60FAB45000506C54F0604DB4100474208010B4200474228009B430047424CE
:20E380008002742612E3B1E57C540F75F004A44443758241F0E57C540F75F002A4F5F0C4C3
:20E3A00054F04408758222F0E5F0C4540FA3F08020900042F0758224F022E57CB40B1474FE
:20E3C000FF12E43AE471B174F21582F074681582F0806C400302E46EB407005029B403004A
:20E3E0005028B4010474FF800274FB12E43AE471B174F31582F0E57CB401047408800274D8
:20E40000281582F0803974228002742071B112E41B802C136817881BA81FC8E57C04540389
:20E4200075F002A4F5F090E41393C0E0E5F00493900022F00582E4F0D0E0900041F0221224
:20E44000E44D90BF34E4F0A3740402898590BF20E4F0A37400F07532037933D2AA301D059B
:20E46000120B728003128E5E2000FD3008057451028D7B2290BF80E0F4540F23FD90E16446
:20E48000301D039000FF93CD0493FC301D057B04023E1522110331FD0131F80100001116CE
:20E4A0008801AFF9D08F030000809F0C800820DA8F0008000004D08F020000809F08800871
:20E4C0002001DA1F12DEEF5301000051D08F0002000052D00081F552FAD08F000000205585
:20E4E000B465B38F0008A50213F8B08F0330A502B18F0001A50212F8B08F0046A502B18F90
:20E500000004A50212F8B08F0004A50295AF8E131BD00150169F080004209118501203311B
:20E520005E00EF00075050D05052112ADB2051E107514DDB2152EF00075252915213121662
:20E54000DB2050E10750F9DB2150EF0007505091501112EC112AA88F000252B052A502B04E
:20E56000A50252B38F00025213F5CA8F0002000052B052A502B0A50252B38F00025212F568
:20E58000B0A50252B38F0001521381B052A502B0A50252B38F00015212F5AA8F000152B07F
:20E5A00052A502EF00075252133895CFEFFE13219052EF36000000DEEF2800000050169FF7
:20E5C0000C000420B0A50252B38F00015213F511BADB2251E10751F9DA5223DB2251E107F5
:20E5E00051F93127FF01000000CF0300000000000000DF15E000FEFFC5150000350A0000BD
:20E60000F53500080200FC03F51503300200F52500010200FC02F51500460200F5250004FD
:20E620000200FC02F51500040200DF8B70FF2080C09772FF17A013000902DF8B70FFFD805E
:20E64000C09772FF17A01100F8021201C055000235100200401D0200C0350002FB03C04566
:20E66000000235100200401D0200C0350002FB02401D0200C0350001D80335100200411D29
:20E680000200C1350001FB02C145000175100200C08BCB03DF8B74FFFD801F9076FFDF8BF5
:20E6A00074FFFD80C201D076D077740612EC6775A00078007976E7F20809B980F97800A685
:20E6C0000008B880FA7800E6B5002B08B880F8E4F8F5D0F539757B04E8B5391A2408F8F5BE
:20E6E00039F5D0D57BF275D00078007976E2F70809B980F9800A757D0C90BF80E030E7AA1A
:20E70000750030AB818881790408C000D9FB7904D0E0B5000D14AA81B5020718D9F28B812B
:20E72000800A757D0C90BF80E030E7D47907750701785574FF585754FF5300555500520029
:20E74000B8012374AA4847440043005545004200E8F4701274AA686764016300556500629E
:20E7600000B85502800A757D0C90BF80E030E7BC7466246630D25F20D65C405AB4CC57B345
:20E78000346620D25130D64E504CB43349C3780675063628250626D338350636F85037B85E
:20E7A0001834C374C9945430D22C20D6294027B4752494FF20D21F30D61C501AB47617C3F0
:20E7C000780575052A98950596400B30D60820D205B41D02800A757D0C90BF80E030E7904F
:20E7E00075F00FE5F0A420D2364034B4E131C5F0702DC5F075F00FA4B42F24C5F0B40D1F0F
:20E8000030D21C75F07774FF8420D2134011B4020EE5F0B41109E4F5F08430D202800A75FA
:20E820007D0C90BF80E030E7B7C350028049D34002804410D702803F20D73C7524167525F7
:20E8400009B35033302130B021402C202402802772245023922A202A02801CB222A2224049
:20E8600016C228D22E82285002800CA02E4008E5244525645E600A757D0C90BF80E030E797
:20E88000A8753838753939A838860176C7E53869F470207938B7C71B7938782F7439C3C87C
:20E8A000231303C404160707253925385005B47B02800A757D0C90BF80E030E7C490BF0091
:20E8C0007404F090BF0474A7F090BF3B7407F07800E4F608B867FBC077C076740302EC67D0
:20E8E000740412EC6790BF007401F0781FE40582F0D8FB90BF007404F0781090BF00E8F05C
:20E9000018758204E8F0187A0412E9AD790512E9B37A0312E9AD790512E9B37A0312E9AD2C
:20E92000790312E9B375821CE8F0781090BF00E0B50036758204E0B40F2F780E7A0412E954
:20E94000AD790512E9BBB900207A0312E9AD790512E9BBB900137A0312E9AD790312E9BB81
:20E96000B9000675821CE080028034B5003190BF007401F0781FE40582F0D8FB90BF00748D
:20E9800004F090BF0474A7F075821AE0F87406D5E0FDE06870517406D5E0FDE06870487566
:20E9A0007D0C90BF81E030E702803C01E0E5822AF58222E8F0058218D9F922E0B500060533
:20E9C0008218D9F722B80A05B4020280F2B808F490BF24E4F090BF21E0B408E890BF2474E4
:20E9E00005F075822180D8900000E4F0A3AA83BABF020583BAFFF47B0078007C018BA0E251
:20EA0000702F74AAFAF2E265027026DCF77C0108B800EC0BBBBF010BBBFFE2900000E0B421
:20EA2000AA0FE4F0A3A883B8BF020583B8FFEF800A757D0490BF80E030E7AC90BF637402BA
:20EA4000F0E4F0F090BF697405F090BF63E0701E90BF68E05470701690BF67E0701090BF7B
:20EA600065E0547F700890BF64E05478600A757D9990BF80E030E7C375A0BF786079637A27
:20EA800000EAF208F27480F3E26A702F18E26A702ADAEE78637401F27A0079627867F30A95
:20EAA000E2541F6A7015EAB410F4F37864E2F5F07865E230F60512EAC78019757D9990BFBA
:20EAC00080E030E7B3800D90BF65E090BF637402F0E4F022740212EC67E57F90BF30E054EB
:20EAE0001E600302EBF1740290BF3FF01582D5E0FA790290BF3FE069600280E71582D9F6FC
:20EB0000740290BF38F00582D5E0FA790290BF38E069600280CD0582D9F690BF80E030E7BC
:20EB20000302EC3978FF793F7AFE7BFFD21090BF327408F090BF307490F090BF3CEAF005DE
:20EB400082EBF090BF36E8F00582E9F090BF30E030E70302EBF1E990BF3715E0F090BF3071
:20EB6000E020E70302EBF110100CD21018B8FF0619B9FF02800DC3EA9402FA400302EB3AE3
:20EB80001B80B77B02E4F520F5217530007A0F8A0190BF327410301101E4F0758233E53084
:20EBA000200108700A7401F0E4800C70027410F0300104241180022410F5307582307474A3
:20EBC000F07470F07582327410F0E4F0D21090BF30E05420701B12EC267016C21012EC2620
:20EBE000B4200EDAAAD211D201753000DB9F02EC3990BF80E030E70790BF30E4F041D4027C
:20EC0000EC3990BF30EAF0F0EBF0630204630304D8F32290BF30EAF0EBF020100663020319
:20EC2000630303D8F12290BF307470F07450F0301002D9FA7460F0E022740112EC67802321
:20EC40009000007800E49328F8A3E583B400F690FFFEE493687002800A757D0590BF80E052
:20EC600020E7D6E57E4487537EF8427E90BF80E030E403437E40437E20E57EF0220D0A0AC2
:20EC800020202020202020202020202020202020202020202020436F7079726967687420DB
:20ECA0003139383820456D756C657820436F72706F726174696F6E0D0A2020202020202043
:20ECC00020202020202020202020202020202020202020202020616C6C207269676874738A
:20ECE00020726573657276656400FFFFFFFFFFFFFFFFFFFFFFFFFFFFFFFFFFFFFFFFFFFFAA
:20ED0000FFFFFFFFFFFFFFFFFFFFFFFFFFFFFFFFFFFFFFFFFFFFFFFFFFFFFFFFFFFFFFFF13
:20ED2000FFFFFFFFFFFFFFFFFFFFFFFFFFFFFFFFFFFFFFFFFFFFFFFFFFFFFFFFFFFFFFFFF3
:20ED4000FFFFFFFFFFFFFFFFFFFFFFFFFFFFFFFFFFFFFFFFFFFFFFFFFFFFFFFFFFFFFFFFD3
:20ED6000FFFFFFFFFFFFFFFFFFFFFFFFFFFFFFFFFFFFFFFFFFFFFFFFFFFFFFFFFFFFFFFFB3
:20FFE000FFFFFFFFFFFFFFFFFFFFFFFFFFFFFFFFFFFFFFFFFFFFFFFFFFFFFFFF030744C906
:00000001FF
